:100000000C9499040C94C1040C94C1040C94C10484
:100010000C94C1040C94C1040C94C1040C94C1044C
:100020000C94C1040C949A050C94BD280C948A3746
:100030000C94C1040C9447350C9485350C94C10480
:100040000C94C1040C94C1040C94C1040C94C1041C
:100050000C94C1044E203B203D203F2041204320F2
:10006000452049204C205A20502052205420562010
:100070005820DA24F424DD24E024E324E824EA24CC
:10008000EE24F124F724F724E324E024CC30CF300D
:10009000D430D930DC30DF30E230E830ED30F430CD
:1000A000F930FC3028312C31313136313A313E31A2
:1000B00044314A314F31533159315D313F32413250
:1000C00043324732473245324B324932000000005A
:1000D0000067582F00000000F567E630C8023200C4
:1000E0002F2CE80310093200802F2C0100000000A3
:1000F0000000000000000000000000000000000000
:100100002ECA7E3BC24CA40B0C49701700000000A5
:1001100043BFA80E0000000080D56610000000005C
:1001200080D0841F0000000031D561100000000065
:10013000C0D665100000000080D4651000000000EB
:1001400080D46510C60232002E2CE8030401320070
:10015000D2052C010006080001FF01010000010684
:10016000090001FF0302010002060A0001FF00006E
:10017000000006060E0000FF0302010005060D0048
:1001800000FF0203000004060C0000FF0302010050
:1001900003060B0000FF040600000706070000FF2F
:1001A00003020100C40D0E0E150F20205475726E4F
:1001B0006967792034783600202020726373747662
:1001C0002E7275002020436865616C694368617216
:1001D00067657200202020207665723A20302E3329
:1001E0003200E60100006F7074696F6E73000100E9
:1001F00001000100010001000A0064000100030089
:1002000008000700070014000700010002000400B6
:1002100010004000000100046D5600206E6F007950
:10022000657300496E6600756E6C696D697465640E
:100230000063025E025902550250024B024602411F
:10024000024E695A6E004C69706F004C696C6F0009
:100250004C6966650050623F004E694D48004E692A
:10026000436400556E6B6E6F776E000098089808B7
:100270006C07102701980898086C0701000298087D
:1002800098086C070100039808DC006C070600045E
:10029000980898086C07030005980898086C0703ED
:1002A0000006980898086C07030007980898086CDF
:1002B00007030001000100010001000000B0041C60
:1002C00007520300000807B0044006E803000008D6
:1002D00007D0079209D60600000000E40C100ED0EB
:1002E00007E40C0000100E0410C409A60E000074F0
:1002F0000E6810B80B0A0F000040066C071405408A
:100300000600004E616D653A0045646974206E61B7
:100310006D653A0053034E03490344033F03310321
:100320002403000020202065646974206E616D65DF
:10033000002020637265617465206E616D650049FF
:10034000643A200049633A200043683A2000563A54
:100350002020004261743A20200025200046554CA0
:1003600020005245564552534520504F4C4152496A
:10037000545900706C656173652063616C696272C9
:10038000617465006265666F72652075736500460D
:10039000756E6374696F6E206E6F7400696D706C3A
:1003A000656D656E746564207965740064656C7450
:1003B0006120543D20006E6F742075736564005495
:1003C0006578743D0064656C746120563D20006D55
:1003D0006178566F75743D006E6F74207573656437
:1003E000006D6F6E69746F72206572726F72007249
:1003F0006561736F6E3A200070726F6772616D2075
:10040000636F6D706C657465002D00546578743D84
:10041000005662616C2E3D00566F7574203D0020C1
:100420006C696D69743D0056696E7075743D007736
:100430006972657320523D00626174742E20523DD2
:100440000020200062200074696D653A2020202081
:1004500020004C696D6974733A20006E2E612E0085
:1004600020202D2D20200043684342426C446946E1
:10047000435374534243684469437943594368443E
:100480006945420064542F6474002D645600562060
:100490006C696D6974009520892099202B21262193
:1004A00034218F218A21D021332201220722642284
:1004B000F0227222000B0C0D64054305FF040000BE
:1004C0000708090A0D6405430516050C05FF04001D
:1004D0000000010203040D640555054D0543053771
:1004E00005FF040000000102030405060D64055524
:1004F000054D05430537052F052005FF0400006560
:10050000646974206261747465727900643E63206A
:100510006379636C6500633E64206379636C650096
:1005200073746F726167652B62616C616E630073D7
:10053000746F7261676500666173742063686172CD
:100540006765006469736368617267650062616C06
:10055000616E6365006368617267652B62616C61DF
:100560006E636500636861726765000106070500D8
:1005700002060708090B0C0D040503000206070814
:10058000090B0C0D0405030006070405000206070D
:1005900008090B0C0D04050300020F0B0C0D0405DC
:1005A0000300020A0E0F0B0C0D040503006578749E
:1005B0002054434F460063617020434F4646006914
:1005C0006E707574205600626174206469736300F4
:1005D000496F75743A20200076616C75653A200089
:1005E000436F6E6E65637420426174746572792125
:1005F0000008090A08090A11060806FF0500005646
:10060000623270696E3A200056623170696E3A202B
:100610000056623070696E3A2000270620060000FE
:1006200076616C75653A0074656D703A20003D0620
:1006300034060000706F696E7420322E00706F698E
:100640006E7420312E005F06520600005F065806C9
:1006500000003330306D4100313030306D410035B5
:10066000306D410006090A0B0C0D0E061E1F2021DD
:1006700022231200B806B206AC06A606A0069A0609
:1006800094068E0688060000566F75743A0056313F
:100690002D363A005662363A20005662353A20002E
:1006A0005662343A20005662333A20005662323A9B
:1006B00020005662313A200056696E3A2000080741
:1006C000FF06F306E706DB06CC06000065787065DA
:1006D00072742044414E474552210063616C696247
:1006E0002D3E554152540074656D702065787465D7
:1006F000726E0049206469736368617267650049BE
:100700002063686172676500766F6C74616765006D
:100710004C074207340700002C071E070000212069
:100720005945532052455345542021002020202074
:10073000204E4F0072657365742064656661756C48
:10074000740063616C6962726174650073657474CE
:10075000696E67730080250000004B000000960062
:100760000000E1000000C2010000007017640007F3
:10077000000C0005007800581B0000080000000372
:1007800000432F6D00AE07A707A10798078F0765E5
:1007900078742E20416463006578742E206465624D
:1007A000006465627567006E6F726D616C006469EC
:1007B0007361626C65640045083A08330829081FB4
:1007C0000813080908FE07F507EB07E407DC07D361
:1007D00007000020202072657365740073706565E2
:1007E000643A2000554152543A200062616C2E2038
:1007F0006572723A006469736368202B3A00696E0F
:10080000707574206C6F773A0063617020434F6697
:10081000663A00432F44206379636C65733A004E57
:10082000694364202D64563A004E694D48202D647A
:10083000563A0064542F64743A00657874726E20DE
:1008400054434F3A00657874726E20543A20202049
:100850000013161817190705061E1F2021222373DF
:1008600020006420006320007265736574696E6700
:1008700020656570726F6D3A00763A20372E312E02
:100880003220000000000000000000000000000016
:10089000040300050000000000000000000000004C
:1008A0000000000000000000000000000001000047
:1008B00000204080000000000001020408102040D9
:1008C00080000001020408102040800000008040E9
:1008D00020100804020100000102040810000202B6
:1008E00002000000000004040404040404040000E6
:1008F00003030303030303030000000101010101DB
:10090000010101000002020202020000390036006B
:100910003300300000003B0038003500320000009A
:100920003A0037003400310087057C105D203C25FB
:10093000773611241FBECFE5D8E0DEBFCDBF10E073
:10094000A0E6B0E0EEE6F3E702C005900D92A63E09
:10095000B107D9F714E0A6EEB0E001C01D92A13AAC
:10096000B107E1F719E0C2E3D9E004C02297FE0124
:100970000E943C39C832D107C9F70E9433370C9422
:10098000B5390C940000CF9388E20E947F38C1E013
:10099000892B09F0C0E089E20E947F38892B11F091
:1009A00080E001C082E0C82B8AE20E947F38892B58
:1009B00011F080E001C084E0C82B8BE20E947F38F8
:1009C000892B11F080E001C088E08C2BCF91089535
:1009D000CF93C82F682F89E10E9410386C2F8AE1CD
:1009E0000E9410386C2F80E20E9410386C2F89E032
:1009F0000E9410386C2F8BE00E9410386C2F80E121
:100A0000CF910C94103808958091FC00882331F028
:100A10008091E6008F5F8093E60002C01092E600AE
:100A20008091FC008A3010F480E001C088E0909151
:100A3000FC00943108F084E09091FC009E3108F0B5
:100A400082E06091E60068238CE20C944938809340
:100A5000FC00089561E068278CE00C94493880E040
:100A60000E94873761E08CE00E94103861E08EE0E0
:100A70000E94103861E08EE10E94103861E08CE243
:100A80000E94103861E08DE00E94103861E08EE035
:100A90000E94103861E08FE00E94103880E00E94D0
:100AA0002A051092FC0020E042E060E187EE90E031
:100AB0000E9494160E9485280E9445230E94A52327
:100AC0000E9409060E94BC070C941C0DCF93C82FEE
:100AD000682F617089E10E9449386C2F62708AE149
:100AE0000E9449386C2F647080E20E9449386C2F54
:100AF000687089E00E9449386C2F60718BE00E9419
:100B000049386C2F607280E1CF910C944938CF92B4
:100B1000EF920F9383E1C82E94E1E92E05E126E1DF
:100B200047E168E187EE90E00E9448170F91EF904F
:100B3000CF9008951F920F920FB60F9211242F930A
:100B40003F934F935F936F937F938F939F93AF9355
:100B5000BF93EF93FF9320910001309101018091A9
:100B6000FE009091FF00820F931F9093FF008093EF
:100B7000FE008091FE009091FF0026E096958795FB
:100B80002A95E1F72091FE003091FF00AC0166E06C
:100B9000440F551F6A95E1F7241B350B3093FF0076
:100BA0002093FE002FB7F8943091FD003E3011F4F1
:100BB0009BBD8ABD3091FD003D30A1F02FBF0E944A
:100BC0000405FF91EF91BF91AF919F918F917F911C
:100BD0006F915F914F913F912F910F900FBE0F90AA
:100BE0001F90189599BD88BDE9CF9FB7F894709371
:100BF0000101609300018093FD008E3019F48FB5E0
:100C0000806804C08D3019F48FB580628FBD9FBF9E
:100C100008951FBC80E18EBD2FB7F89480E091E06D
:100C200097BD86BD2FBF8EB5887F8EBD8EB5816086
:100C30008EBD89B7846089BF08958E3019F48FB551
:100C40008F7704C08D3019F48FB58F7D8FBD0895D7
:100C50008091030190910401A0910501B0910601DA
:100C6000892F9A2FAB2FBB27A7FDBA950895109215
:100C70000A01109209018617970768F480E090E452
:100C8000A0E0B0E08093030190930401A0930501DC
:100C9000B093060108C01092030110920401109253
:100CA0000501109206018091030190910401A09129
:100CB0000501B0910601BA2FA92F982F882780939C
:100CC000030190930401A0930501B093060181E014
:100CD000809302010895CF93DF93EC01C13080E649
:100CE000D80770F4C13080E4D80760F48EE00E9429
:100CF0001D0660E08EE00E944938BE018DE00CC008
:100D0000C0E0D0E68DE00E941D0661E08DE00E940B
:100D10004938BE0170548EE0DF91CF910C94F505F7
:100D200090930A01809309016CEB76E680E00E94C3
:100D3000BE0C90930801809307010895CF93C82FAC
:100D4000882319F080E00E94AB0661E06C278EE1F9
:100D5000CF910C944938CF93DF93C82F882319F093
:100D600080E00E949E068DE00E941D0660E08DE0FE
:100D70000E9449388EE00E941D0660E08EE00E94CD
:100D800049381092020161E06C278FE00E944938D7
:100D9000CC2361F080E00E949508EC0186E00E947F
:100DA0009508BE01DF91CF910C943706DF91CF916A
:100DB00008950F931F9380910201882309F474C052
:100DC00080E00E949E0820910701309108012817B9
:100DD000390730F480E00E94AB061092020164C033
:100DE00082E00E949E084091090150910A0160E052
:100DF00070E00091030110910401209105013091F0
:100E00000601481B590B61097109E4E0440F551FA5
:100E1000661F771FEA95D1F7040F151F261F371F8E
:100E20000093030110930401209305013093060100
:100E30008091030190910401A0910501B0910601F8
:100E4000B7FF08C01092030110920401109205012F
:100E5000109206018091030190910401A091050177
:100E6000B09106010197A046B10560F080E090E0E6
:100E7000A0E6B0E08093030190930401A0930501E4
:100E8000B09306018091030190910401A0910501A6
:100E9000B0910601892F9A2FAB2FBB27A7FDBA95DA
:100EA0001F910F910C946B061F910F910895BC0137
:100EB0008EE00C94F5058770806287B90895CF9312
:100EC000DF9390916600891721F180936600C8B383
:100ED00090E2899F90011124CF71C22B98B3EFEC5F
:100EE000F8E0E4912AB3DE2FD095D2232AB38150C3
:100EF000823050F0892F8F71806C88BBE22BEABB67
:100F00008AE090E00E94D4378FB7F894C8BBDABB70
:100F10008FBFDF91CF91089594B125B135E0839FC4
:100F2000F0011124EA5AFE4FE491F0E0EE0FFF1FAA
:100F3000EC54FE4F892F90E0922B9183808308958B
:100F400010920B01E5E5F1E084910E945B07E4E576
:100F5000F1E084910C945F07369A08950E940B2368
:100F60009093D3018093D2010E945B239093D5018B
:100F70008093D4010C948D0C60E08FE10E9449387D
:100F800060E08FE10E94103861E081E00E9410383B
:100F900061E082E00E94103861E083E00E94103836
:100FA00087E886B90C94A007CF93DF93E0910B01FB
:100FB0008E2F90E025E0E29FF0011124E85AFE4FC9
:100FC000E491EE2321F0C0913C02C17001C0C0E069
:100FD00025E0289FF001299FF00D1124EC5AFE4FC7
:100FE0008491C11109C020915B0330915C03232BD4
:100FF00021F0873011F4C1E085E00E945F07E091A5
:101000000B01EF5F85E0E89FF0011124EB5AFE4FE2
:1010100084910E945B078CE390E00E94D4370E9489
:10102000AC073699FECFD0910B0181E08D0F0E9465
:101030008C0725E0D29FF0011124EB5AFE4F8491DA
:101040000E945B078CE390E00E94D4370E94AC07BB
:101050003699FECFC11104C080910B010E948C070C
:10106000E0910B01EF5F85E0E89FF0011124E95A60
:10107000FE4FE491E1110E94D90680910B018E5F31
:10108000803118F480930B0102C010920B010E9472
:10109000A708882341F080910B01811104C0DF91E2
:1010A000CF910C94AE07DF91CF9108950C94A007D7
:1010B000CF93DF930E94900AC0912201D091230127
:1010C0008091220190912301C817D90719F40E9439
:1010D000D407F6CFDF91CF910895CF92DF92EF92B0
:1010E000FF92CF93DF93EC010E94E1286B017C011A
:1010F000CC0EDD1EE11CF11C0E94D4070E94E128E9
:101100006C157D058E059F05B8F3DF91CF91FF909B
:10111000EF90DF90CF900895E82FF0E0EE0FFF1FE3
:10112000EA52FE4F808191810895E82FF0E0EE0FA2
:10113000FF1FE459FE4F808191810895E82FF0E070
:10114000EE0FFF1FEC54FE4F808191810895809136
:101150003E02089580912201909123010895E82F85
:10116000F0E0EE0FFF1FEC5DFE4F8081918108954E
:10117000262F613110F4423040F021E030E0FC01D4
:101180003383228331832083089550E0BA01620FB4
:10119000711D620F711D660F771F660F771F6E5FDF
:1011A0007F4F44E050E00C947039282FCA01213160
:1011B00088F4623078F470E0620F711D620F711D67
:1011C000660F771F660F771F6E5F7F4F44E050E01A
:1011D0000C948E390895FF920F931F93CF93DF9352
:1011E00000D000D0CDB7DEB70CEC10E0F12CF80148
:1011F000459155916591749149835A836B837C83A2
:10120000AE014F5F5F4F60E08F2D0E94D508F8015F
:101210003496459155916591749149835A836B83B6
:101220007C83AE014F5F5F4F61E08F2D0E94D50838
:10123000F394085F1F4F81E1F812D9CF0F900F9000
:101240000F900F90DF91CF911F910F91FF90089514
:10125000E82FF0E0EE0FFF1FE459FE4F20813181AF
:10126000EEEFE80FE53170F4F0E0ED58FF4F8081CC
:10127000882319F0813061F405C081E02333310502
:1012800040F404C081E0293E334018F480E0089522
:1012900081E00895CF93C0E08EE18C0F0E94280971
:1012A000882329F0CF5FC630B9F786E001C08C2FC4
:1012B000CF910895209198013091990180910C016E
:1012C00090910D01A0910E01B0910F01820F931F1B
:1012D000A11DB11D80930C0190930D01A0930E01EF
:1012E000B0930F01089560910C0170910D018091F0
:1012F0000E0190910F012DE730E040E050E00E9498
:10130000F938BB27A52F942F832F08958091920140
:1013100090919301089580914A0190914B01039718
:1013200050F08091500190915101039720F083E09B
:1013300090E00C94480E80E0089590E0880F991F8B
:10134000FC01E459FE4F208131816217730718F4C4
:10135000261B370B04C0AB01421B530B9A01FC0147
:10136000EC5DFE4F2730310518F01182108206C067
:10137000208131812F5F3F4F31832083FC01E4596D
:10138000FE4F718360830895AF92BF92CF92DF9238
:10139000EF92FF920F931F93CF93DF931F92CDB7DE
:1013A000DEB700916C0110916D0160917C0170912C
:1013B0007D0180917E0190917F016817790728F463
:1013C0009C01261B370BB90102C0681B790B8EE10B
:1013D0000E949D0960917E0170917F018091800142
:1013E000909181016817790728F4FC01E61BF70B3F
:1013F000BF0102C0681B790B8FE10E949D0952E872
:10140000E52E51E0F52E90E2F701619171917F0197
:10141000892F99830E949D0999819F5F9432A1F73A
:101420000E944A09F82E80E0A12CB12C8F1569F09A
:10143000EEE1E80FF0E0EE0FFF1FE459FE4F2081D0
:101440003181A20EB31E8F5FF1CFB50182E10E9400
:101450009D09A114B10449F0A016B10650F49801F9
:101460002A193B09293E334020F0580110E0F12CA5
:1014700001C012E1B50183E10E949D096F2D70E06A
:1014800085E10E949D09612F70E084E10E949D0921
:101490000E9473098C010E944C23882329F0E0905C
:1014A0007201F09073010BC00E94FC22882329F086
:1014B000E0907001F090710102C0E12CF12CB701B5
:1014C00086E10E949D09B80188E10E949D0997016B
:1014D000D5010E94A83830E1C32E37E2D32EE12C8B
:1014E000F12CA70196010E94F938B90187E10E9409
:1014F0009D099801D5010E94A838A70196010E9474
:10150000F938B90189E10F90DF91CF911F910F91C7
:10151000FF90EF90DF90CF90BF90AF900C949D091B
:1015200010923D0210923C02E8EFF1E0119211920C
:101530001192119282E0EC33F807C1F708951092EE
:101540001F0110921E0110921A0110921B0110929D
:101550001C0110921D011092160110921701109299
:10156000180110921901109221011092200110927D
:101570001501109214010E94E128609310017093EC
:10158000110180931201909313010895E4E2F1E0B8
:101590001192119281E0EC36F807D1F708950E947C
:1015A000900A0C94C60A1092230110922201109204
:1015B0000C0110920D0110920E0110920F010E9469
:1015C00056080E94CF0A0E949F0AECE6F1E01192B1
:1015D000119281E0E43BF807D1F7089580913E0233
:1015E00081110AC081E00E942A050E94D30A81E08D
:1015F00080933E020C945808089510923E0280E0B9
:101600000C942A052091B6013091B7018091B40164
:101610009091B5018217930718F4281B390B02C06B
:1016200020E030E081E0293E334008F480E0089576
:101630008F929F92AF92BF92CF92DF92EF92FF92E2
:10164000CF93DF93CDB7DEB728970FB6F894DEBF00
:101650000FBECDBFF82E5B0140E0682FCE0105968E
:101660000E94B80841E06F2DCE0101960E94B80893
:101670002B813C8140E050E0CF80D884E12CF12CDC
:101680002C193D094E095F09B50180E090E08D807D
:101690009E80A12CB12C681979098A099B090E94A6
:1016A000C93829813A8140E050E0281939094A09AE
:1016B0005B090E941B392C0D3D1D4E1D5F1D57FF00
:1016C00003C020E030E0A901C90128960FB6F894C4
:1016D000DEBF0FBECDBFDF91CF91FF90EF90DF90C7
:1016E000CF90BF90AF909F908F9008950F931F93CE
:1016F000CF93DF93C1E020919401309195018091C7
:101700001A0190911B01A0911C01B0911D01223181
:10171000310531F0C0E02091B4013091B50104C031
:101720002091920130919301820F931FA11DB11D51
:1017300080931A0190931B01A0931C01B0931D018B
:101740002091C2013091C30180911601909117013F
:10175000A0911801B0911901820F931FA11DB11D15
:101760008093160190931701A0931801B09319016B
:1017700080911E0190911F01019690931F0180930B
:101780001E010E94E1280091100110911101209189
:10179000120130911301601B710B820B930B6136A8
:1017A0007A4E8105910508F479C0809120019091CD
:1017B00021010196909321018093200120911E0127
:1017C00030911F0140E050E060911A0170911B01BF
:1017D00080911C0190911D010E94F938890110929D
:1017E0001A0110921B0110921C0110921D01C111CF
:1017F00005C0B90180E00E94180B8C01C091A201C4
:10180000D091A3010C171D0720F0B8018BE10E94B5
:101810009D09B8016C1B7D0B8AE10E949D092091F6
:101820001E0130911F0140E050E06091160170915F
:10183000170180911801909119010E94F9381092B6
:101840001601109217011092180110921901B90196
:1018500087E00E94180B209114013091150190939C
:10186000150180931401BC01621B730B8CE10E9473
:101870009D0960911E0170911F018DE10E949D09DB
:1018800010921F0110921E010E94E1286093100126
:10189000709311018093120190931301DF91CF9106
:1018A0001F910F910895FF920F931F93CF93DF9392
:1018B00080912201909123010196909323018093BE
:1018C000220108EF11E0C6EDD1E0F12CF8016191A1
:1018D0007191819191918F0120913C0230913D0253
:1018E00040E050E00E94F93829933993B9018F2DD7
:1018F0000E94180BBC018F2D0E949D09F394F1E109
:10190000FF12E4CF0E94C4090E94F633DF91CF9109
:101910001F910F91FF900C94900ACF93DF93E4EB0B
:10192000F1E0C8EFD1E02191319188819981AA81BC
:10193000BB81820F931FA11DB11D89939993A99318
:10194000B99381E0E63DF80771F780913C029091F0
:101950003D02019690933D0280933C020E94760BDB
:1019600080913C0290913D028436910521F4DF91F3
:10197000CF910C94530CDF91CF9108958F929F9249
:10198000AF92BF92CF92DF92EF92FF92CF93DF930D
:10199000CDB7DEB728970FB6F894DEBF0FBECDBF28
:1019A000F82E5B0140E0682FCE0105960E94B80832
:1019B00041E06F2DCE0101960E94B80829813A813D
:1019C00040E050E0CD80DE80E12CF12C2C193D0967
:1019D0004E095F09B50180E090E08F809884A12CCA
:1019E000B12C681979098A099B090E94C9382B8191
:1019F0003C8140E050E0281939094A095B090E94FE
:101A00001B392C0D3D1D4E1D5F1D57FF03C020E0EF
:101A100030E0A901C90128960FB6F894DEBF0FBEC9
:101A2000CDBFDF91CF91FF90EF90DF90CF90BF902F
:101A3000AF909F908F9008950C94D30A462FE82F73
:101A4000F0E0EE0FFF1FE459FE4F208131818250FC
:101A5000853130F4E82FF0E0ED58FF4F608101C090
:101A600061E0C9010C946915825E0C94950880911F
:101A70006502089580916302811113C00E94A70836
:101A8000882381F00E94AA0820913F0230914002F1
:101A9000821B930B9C0181E02530310518F080E01A
:101AA000089581E008950F931F93CF93DF9310E083
:101AB000CFEFDFEF00E080916502181760F4812F0F
:101AC0000E94340D8C179D0710F0CE0101C0012F2C
:101AD0001F5FEC01F0CF802FDF91CF911F910F910D
:101AE0000895CF93DF9390916302911104C0DF9129
:101AF000CF910C94340D90914902C82FD0E09923D6
:101B000091F00E94340DCC0FDD1FFE01E65BFD4F0E
:101B1000CA5ADD4F2081318148815981241B350B00
:101B2000280F391F07C0FE01EE0FFF1FE65BFD4FB8
:101B300020813181C901DF91CF910895CF93C82FC2
:101B400080916302882341F0C11106C00E94AA0857
:101B50009093400280933F02C09363020E94E12869
:101B60006093410270934202809343029093440237
:101B70000E94C60A80916202811104C08C2FCF910D
:101B80000C946605CF910895EF92FF920F931F93E7
:101B9000CF93DF9381E00E94E80485E10E949508DD
:101BA0008093650206E512E03AE4E32E32E0F32E7C
:101BB000C0E0D0E08091650290E0C817D9076CF4CE
:101BC0008C2F0E94340DF801819391938F01F701BE
:101BD000819391937F012196EDCF10926302109231
:101BE000620280E00E949E0D1092400210923F021D
:101BF000109241021092420210924302109244024B
:101C0000DF91CF911F910F91FF90EF90089580E0A9
:101C10000E949E0D81E08093620208950E94070E4B
:101C200080E00C94E804FF920F931F93CF93DF930F
:101C3000809164020E94710DEC01F12C01E010E032
:101C400080916502F816E8F48F2D0E94710DAC01A9
:101C500080916302802321F0C417D50778F40DC06A
:101C60002091590330915A032F5F3F4F36952795A6
:101C70002C0F3D1F2417350708F4102B000FF39489
:101C8000DFCF812FDF91CF911F910F91FF900895AA
:101C90001F93CF93DF93EC0110E08091650218173A
:101CA00048F48EE1810F0E94AF088C179D0720F049
:101CB0001F5FF3CF81E001C080E0DF91CF911F91E2
:101CC0000895BF92CF92DF92EF92FF920F931F93EE
:101CD000CF93DF938AE090E00E94480E882309F4B6
:101CE00060C00E94530D809364020E94340D8C01E9
:101CF00062E084E792E00E9437190817190748F15B
:101D00007AE4E72E72E0F72EE6E5CE2EE2E0DE2E54
:101D1000C0E0D0E0BB24B3948091650290E0C81786
:101D2000D907CCF48C2F0E94340DF7018193919345
:101D30007F01F601819391936F01801B910B20919C
:101D4000590330915A032817390708F4B12C21960A
:101D5000E3CFBB24B394109249020E94E128609320
:101D60004502709346028093470290934802BB203D
:101D700059F0DF91CF911F910F91FF90EF90DF907D
:101D8000CF90BF900C94070E0E94130EDF91CF915D
:101D90001F910F91FF90EF90DF90CF90BF900C9428
:101DA0009E0DDF91CF911F910F91FF90EF90DF90EB
:101DB000CF90BF900895CF9380914902811119C0AF
:101DC00081E080934902809164020E94340DC0E05A
:101DD00080916502C81768F48C2F0E94340DEC2F97
:101DE000F0E0EE0FFF1FEA5AFD4F91838083CF5F33
:101DF000EFCFCF9108950F931F930E94E128009198
:101E00004502109146022091470230914802601B22
:101E1000710B820B930B28EE33E040E050E00E9400
:101E2000F938C9011F910F91089583E090E00E9455
:101E3000480E8823C9F080916302811103C00E947B
:101E4000610E12C00E94DB0E0E94130E90E080957E
:101E500090952091630230E082239323892B81F4B3
:101E60000E94FB0E4F9760F40E943A0D882311F0F8
:101E700082E00895809162028823D1F381E0089581
:101E800080E00E949E0DF0CF1F93CF93DF93EC0173
:101E900010E080916502181780F4812F0E94340DA4
:101EA0008C179D0710F081E009C0812F0E94710DF1
:101EB0008C179D07C0F71F5FECCF80E0DF91CF91BB
:101EC0001F9108951F93CF93DF93EC0110E0809151
:101ED0006502181780F4812F0E94340DC817D907A6
:101EE00010F081E009C0812F0E94710DC817D90739
:101EF000C0F71F5FECCF80E0DF91CF911F91089575
:101F000060916502662329F070E00E94E538CB01FC
:101F1000089580E090E008950E9410120E945A1FD8
:101F200085E00E947F310E94D12988E00C947F31A6
:101F30000E9410120E945E1F86E00E947F310E9464
:101F4000D12988E00C947F31E0916602F09167021C
:101F500085919491FC010994E0916602F0916702E9
:101F6000329685919491FC010994E0916602F0917A
:101F70006702349685919491FC010994CF93DF9385
:101F80001F92CDB7DEB7811107C00E943B1E0E9491
:101F9000AC0F0E94980F0FC0813059F469830E94E2
:101FA0003B1E0E94AC0F6981611105C00E948C0F1D
:101FB00002C081E001C080E00F90DF91CF910895D1
:101FC000BF92CF92DF92EF92FF920F931F93CF9326
:101FD000DF938C01C62E0E94A40F0E941D1E0E943A
:101FE000F6290E941012F12C82E0D82EC0E0D0E039
:101FF000EE24E3940E946431811106C0F801EF0DD4
:10200000F11D84910E942C200E949F11B82E84E023
:10201000B81209C0EF2DF0E03196E00FF11FE49106
:10202000E11123C005C082E0B81202C0F110FA9499
:10203000EE2081F00E94002AD82E6C2D0E94BE0F47
:10204000E82E882339F00E94AA08C817D90779F426
:10205000E11003C0C11016C0E12C81E0B812CACF54
:102060000E943B1E0E94AC0F0DC0F394E1CF0E9472
:10207000AA08EC010E94B50FD82E6C2D0E94BE0F4D
:10208000E82EE6CF8D2DDF91CF911F910F91FF901C
:10209000EF90DF90CF90BF90089560E088E692E0E7
:1020A0000E947E1887FD0AC0811102C00C94E92E9F
:1020B000992787FD909501970C94FE2408950E941E
:1020C0002F050E9469320E942A2F64ED71E084EC92
:1020D00091E00E943D1F88EE93E00E946D0868EB3E
:1020E00071E08AEA91E00E943D1F88EE93E00E9431
:1020F0006D0880E00C94E73662EE71E088E692E0CD
:102100000E9490178CE890E0909369028093680297
:10211000ECE6F2E08081805E80830895FC012481FA
:102120002052621710F40C948317862F90E0821BC4
:1021300091090E94FE196EE00C945213CF93DF9325
:10214000EC010E9408128B819C810E944F130E9417
:102150000C126A8188819981DF91CF910C94E712EA
:10216000FC0187818F3118F48F5F87830895868102
:102170008F5F86830895FC018781882319F0815041
:102180008783089586818150868308950F931F93D6
:10219000CF93DF93FC01C681D0E06D2F80E00E94D9
:1021A000021210E11C0F01E00C0F8C2F0E94A013F3
:1021B000011711F0C02FF7CFDF5FD23011F0C12F20
:1021C000ECCFDF91CF911F910F9108951F93CF9383
:1021D000DF93EC0187EE90E00E9475171FEF8E8170
:1021E000181721F0CE010E94C6101E818F81682F22
:1021F00070E094E0759567959A95E1F78F700E946D
:1022000002120E949F11823049F0843019F081300F
:1022100049F413C0CE010E94B010E1CFCE010E945C
:10222000BB10DDCF8830D9F68D81E881F981E80FC8
:10223000F11D8F819E81890F8083DF91CF911F9146
:102240000895FC0171836083428334832383158264
:1022500080E2868317820895CF93DF93EC0187EEA7
:1022600090E00E9475170E941012CE010E949E10ED
:1022700061E08D810E9402120E949F118230B1F0B4
:10228000843041F08130C1F487EE90E00E946E17F7
:1022900080E026C04D81242F30E08A8190E00197B4
:1022A000281739072CF74F5F4D83E2CF8D818823A4
:1022B000F9F281508D83DCCF8830D1F682E00E9424
:1022C000F111823048F083E00E947F3187EE90E088
:1022D0000E946E1781E004C0CE010E94E610C3CFB9
:1022E000DF91CF9108950C94C304E0917202F0E065
:1022F000EE0FFF1FE251FE4F859194910895CF9309
:10230000DF93D82F0E94C304C82F8D1741F082E3BA
:1023100090E00E946D080E94C304DC2FF5CF10925C
:1023200072021092710280937302882319F080E088
:102330000E94883180917302DF91CF910895FF92BE
:102340000F931F93CF93DF93C0E0D0E0F12C0AEFFF
:1023500010E040917202242F30E0220F331FF90168
:10236000E65FFD4F65917491C8010E94E5386F5F8B
:102370007F4FC617D707A8F40E94C304F82E81E048
:1023800090E00E946D0880917302F81641F08F2D45
:10239000DF91CF911F910F91FF900C947F112196A7
:1023A000D8CFFF20B1F0509171025F5F509371025E
:1023B000F901E450FE4F85919491252F30E02817C4
:1023C000390738F0463018F44F5F4093720210928C
:1023D000710280917302DF91CF911F910F91FF9055
:1023E0000895CF93DF93D82FC09173020E949F115D
:1023F000909172029D1711F08C17C1F3892FDF9114
:10240000CF910895462F682F87EE90E00C945F16C9
:1024100060E080E00C94021261E080E00C94021213
:1024200087EE90E00C945816CF93DF93FC01DB010C
:102430008C91882389F0C081D181488380819181EA
:102440000196918380838C9181508C93882321F015
:102450000190F081E02D1082DF91CF910895BF921D
:10246000CF92DF92EF92FF920F931F93CF93DF9360
:10247000EC018B017A014115510501F1CA010E945D
:102480004939F8019081B82E981708F4B92ECB2C51
:10249000D12CA601B701888199810E9452392881E7
:1024A00039812C0D3D1D39832883F80180818B19DA
:1024B0008083882319F0E881F9811082DF91CF9120
:1024C0001F910F91FF90EF90DF90CF90BF900895F4
:1024D000EF92FF921F93CF93DF9300D000D0CDB740
:1024E000DEB77C01CA014B835C8369837A830E94D7
:1024F0005429182F69817A81DB018C914B815C8191
:10250000811768F44FE3C7010F900F900F900F9061
:10251000DF91CF911F91FF90EF900C941412F7016F
:1025200020813181210F311D31832083DB018C918A
:10253000811B8C93882321F00190F081E02D108283
:10254000F9012AE030E0112369F0CA01B9010E94C3
:10255000E538405DBAE06B9F401911244293115059
:10256000AB01F1CF0F900F900F900F90DF91CF91B3
:102570001F91FF90EF9008950F931F93CF93DF93D8
:10258000CDB7DEB72B970FB6F894DEBF0FBECDBF29
:102590008E010F5F1F4F1A87098727E02B87AC0139
:1025A000BE01655F7F4FCE0109960E946812B80197
:1025B00087EE90E00E947E372B960FB6F894DEBF30
:1025C0000FBECDBFDF91CF911F910F9108950F9353
:1025D0001F93CF93DF93CDB7DEB761970FB6F89413
:1025E000DEBF0FBECDBF0097D1F0613108F060E1D2
:1025F000062F10E0A801BC01CE0101960E946139AE
:10260000E1E0F0E0EC0FFD1FE00FF11F1082BE01D2
:102610006F5F7F4F87EE90E00E947E3701C080E0C1
:1026200061960FB6F894DEBF0FBECDBFDF91CF919C
:102630001F910F9108950F931F93CF93DF93CDB701
:10264000DEB761970FB6F894DEBF0FBECDBF00971F
:10265000D1F0613108F060E1062F10E0A801BC0163
:10266000CE0101960E945239E1E0F0E0EC0FFD1F2F
:10267000E00FF11F1082BE016F5F7F4F87EE90E089
:102680000E947E3701C080E061960FB6F894DEBFED
:102690000FBECDBFDF91CF911F910F91089560E1E3
:1026A0000C941B13CF92DF92EF92FF920F931F9324
:1026B000CF93DF93CDB7DEB762970FB6F894DEBF46
:1026C0000FBECDBF009719F1613108F060E16C01D8
:1026D0008E010F5F1F4F78018E2D801B861768F4C7
:1026E000C6016A8B0E948039F70181937F01FFEF59
:1026F000CF1ADF0A6A898111EFCFF801E60FF11DC9
:102700001082B80187EE90E00E947E3701C080E021
:1027100062960FB6F894DEBF0FBECDBFDF91CF91AA
:102720001F910F91FF90EF90DF90CF900895882335
:1027300019F08FE192E002C08BE192E00C944F130C
:10274000682F87EE90E00C948037CF93DF93D82FDB
:10275000C0E0CD1729F080E20E94A013CF5FF9CF2F
:102760008C2FDF91CF91089580E10C94A513CF9326
:10277000DF931F92CDB7DEB7682F64303CF080E264
:1027800069830E94A01369816150F7CF83E292E0D0
:102790000F90DF91CF910C941B136AE00E94D938FF
:1027A00080E3890F0C94A013DF92EF92FF920F93B6
:1027B0001F93CF93DF93EC01F62ED42E16160CF058
:1027C00086C068EE73E00E94E5388B01CB010E9461
:1027D000542924E0E22EE80EEF142CF480E20E944B
:1027E000A013FA94F9CFFE14D4F0D11018C0CE0182
:1027F0000E945429182FFA941F1524F480E20E9495
:10280000A013F9CFCE010E94BC128DE6DF91CF91CB
:102810001F910F91FF90EF90DF900C94A0132E2D3D
:10282000332727FD3095245031094F2D552747FD7B
:1028300050954217530754F48F2DDF91CF911F917C
:102840000F91FF90EF90DF900C94B713C8010E9496
:10285000BC12CE0168EE73E00E94E538EC011F2D3A
:102860001E1993E0F92EF10E84E0810F18161CF466
:102870008EE20E94A01302E0010F1F1444F4CE0167
:1028800064E670E00E94E538862F0E94CD13CE01E9
:1028900064E670E00E94E538EC011F5F10163CF41E
:1028A0006AE070E00E94E538862F0E94CD13111671
:1028B00074F4CE016AE070E00E94E538DF91CF91B8
:1028C0001F910F91FF90EF90DF900C94CD13DF914B
:1028D000CF911F910F91FF90EF90DF900895EF92AD
:1028E000FF920F931F93CF93DF93EC01F62E1616F2
:1028F0000CF058C064E670E00E94E5388B01CB0113
:102900000E94542933E0E32EE80EEF142CF480E209
:102910000E94A013FA94F9CF2E2D332727FD30956E
:10292000235031094F2D552747FD50954217530726
:102930004CF48F2DDF91CF911F910F91FF90EF906D
:102940000C94B713C8010E94BC12CE0164E670E07B
:102950000E94E538EC010F2D0E1912E0100F83E0F4
:10296000800F18161CF48EE20E94A013FF24F3942B
:10297000F00E111644F4CE016AE070E00E94E538D2
:10298000862F0E94CD131F146CF4CE016AE070E014
:102990000E94E538DF91CF911F910F91FF90EF904A
:1029A0000C94CD13DF91CF911F910F91FF90EF9079
:1029B0000895BF92CF92DF92EF92FF920F931F93F1
:1029C000CF93DF938C01D62EB42EC22E16169CF513
:1029D0002111DA94C8010E945429C82FD0E0ED2CAF
:1029E000FF24E7FCF094CE15DF052CF48B2D0E941C
:1029F000A013DA94F4CFCC2019F08DE20E94A0133A
:102A0000EC16FD0664F48D2DDF91CF911F910F918F
:102A1000FF90EF90DF90CF90BF900C94B713C80158
:102A2000DF91CF911F910F91FF90EF90DF90CF90AA
:102A3000BF900C94BC12DF91CF911F910F91FF902A
:102A4000EF90DF90CF90BF90089520E00C94D914C0
:102A5000CF93DF936CE370E00E94E5389B01EC01BB
:102A600040E363E0C9010E9425158AE30E94A01398
:102A700040E362E0CE01DF91CF910C94251540E256
:102A80000C942515292F221F2227221F19F091951A
:102A90008195910940E20C94D914161634F46150D2
:102AA0000E946F1483E40C94A0130895161634F456
:102AB00061500E943F1585E20C94A0130895633085
:102AC0003CF062500E943F1588E192E00C944F1355
:102AD0000895CF93DF93C62F141674F56FEF640F2C
:102AE000C23081F030F4CC23B1F0C130B9F4D6E576
:102AF00016C0C43061F068F0C53081F40E94421500
:102B000085E516C0642FDF91CF910C944D15D4EF5D
:102B100003C06EEF640FD1E440E002C0D5E541E0B0
:102B20000E94D4138D2F0E94A013C33029F488E68D
:102B3000DF91CF910C94A013DF91CF910895462F90
:102B400063E00C946915462F60E00C946915462FDC
:102B500061E00C946915462F64E00C946915CF93DD
:102B6000DF93EC0160E08E810E94493881E090E0C3
:102B70000E94D43761E08E810E94493881E090E064
:102B80000E94D43760E08E810E94493884E690E04C
:102B9000DF91CF910C94D437CF92DF92EF92FF92D6
:102BA0000F931F93CF93DF937C01C0E0D0E0C62E3C
:102BB000D12C87010C0F1D1F61E0F80187810E9455
:102BC0001038B6010C2E02C0759567950A94E2F78D
:102BD0006170F80187810E9449382196C430D1057F
:102BE00041F7C701DF91CF911F910F91FF90EF90B7
:102BF000DF90CF900C94AF15CF92DF92EF92FF92BF
:102C00000F931F93CF93DF937C01C0E0D0E0C62EDB
:102C1000D12C87010C0F1D1F61E0F80187810E94F4
:102C20001038B6010C2E02C0759567950A94E2F72C
:102C30006170F80187810E9449382196C830D1051A
:102C400041F7C701DF91CF911F910F91FF90EF9056
:102C5000DF90CF900C94AF151F93CF93DF93EC01CF
:102C6000162F642F8C810E9449388D818F3F19F077
:102C700060E00E9449388F85612F84FF06C0CE0135
:102C8000DF91CF911F910C94FC1570E084E0759555
:102C900067958A95E1F7CE010E94CC15612FCE0190
:102CA000DF91CF911F910C94CC1540E00C942C1621
:102CB00061E00E94551680ED97E00C94D437CF93D5
:102CC000DF93CDB7DEB728970FB6F894DEBF0FBEFF
:102CD000CDBF28E0EBE6F0E0DE01119601900D9209
:102CE0002A95E1F7FC012389421710F04FEF420FBC
:102CF000FE013196E40FF11DE40FF11D2081260F36
:102D00002068622F28960FB6F894DEBF0FBECDBFA5
:102D1000DF91CF910C945516FC016089262F246019
:102D2000208B6C600C945516CF93DF93EC014230EE
:102D300018F08F8588608F874B8B1C8A222329F09F
:102D4000413019F48F8584608F8780E593EC0E9471
:102D5000D43760E08C810E94493860E08E810E9407
:102D600049388D818F3F19F060E00E9449386F85A6
:102D700064FD1DC063E0CE010E94CC1584E991E1A1
:102D80000E94D43763E0CE010E94CC1584E991E122
:102D90000E94D43763E0CE010E94CC1586E990E012
:102DA0000E94D43762E0CE010E94CC1516C060624A
:102DB000CE010E94551684E991E10E94D4376F85B7
:102DC0006062CE010E94551686E990E00E94D437D9
:102DD0006F856062CE010E9455166F856062CE01DC
:102DE0000E94551684E0888BCE010E948C16CE017D
:102DF0000E94581682E0898B66E0CE01DF91CF9168
:102E00000C9455166F927F928F92AF92CF92EF9261
:102E10000F931F93CF93DF93CDB7DEB73C01162FEF
:102E2000842F5D854E853F859889F30184832583B2
:102E30000683E782C086A1868286538744873587CA
:102E4000968761E00E941038F30185818F3F19F069
:102E500061E00E94103861E0F30186810E94103821
:102E6000112319F0F301178603C080E1F30187876E
:102E700020E041E060E1C301DF91CF911F910F910C
:102E8000EF90CF90AF908F907F906F900C949416AE
:102E90008F92AF92CF92EF920F93DC0113961C9218
:102EA0001E921297E2E9F0E0ED93FC931F921F92BD
:102EB0001F921F928C2CAE2CC02EE22E042F2FEFCF
:102EC000462F61E00E9402170F900F900F900F9015
:102ED0000F91EF90CF90AF908F900895FC01608993
:102EE0006E7F608B68600C945516FC016089262FFC
:102EF0002160208B69600C94551641E00E942C16CD
:102F000081E090E00895FC0127818085E22FF82F71
:102F1000E60FF11DE60FF11D859194910C944F136E
:102F20000F931F93CF93DF93EC018B01CB010E9492
:102F30000E29682FCE010E94F3178AE990E0998349
:102F4000888318870F83DF91CF911F910F91089588
:102F5000DF92EF92FF920F931F93CF93DF93EC01D9
:102F6000F62E69871A8681E08D8382E0D82EEE24C2
:102F7000E3948E01075F1F4F0E949F11482F8230FC
:102F800011F0843061F4E881F9810280F381E02D51
:102F90006F2DCE010995F986DA86ED8204C0813065
:102FA00089F0883079F0C8010E94E5298111ED820D
:102FB0008D81882319F0CE010E9420188A858F5FA9
:102FC0008A87DACF8FEF898781E08E838D834830BF
:102FD00009F080E0DF91CF911F910F91FF90EF906A
:102FE000DF9008950895FC0180EA90E0918380834A
:102FF00012821382648381E0858386830895FC01B5
:103000002281211103C081E082830895438130E051
:10301000240F311D848190E001972817390714F49B
:103020004F5F43830895FC018281882319F081500A
:10303000828308958381882311F0815083830895CA
:103040001F93CF93DF93EC0110E0612F80E00E948B
:10305000021280E20E94A013E881F9816B81610F66
:103060000190F081E02DCE0109950E94B4131F5FFD
:10307000123059F76A8180E00E9402128EE30E94AA
:10308000A0136A818FE00E9402128CE30E94A013B9
:103090001D82DF91CF911F9108950F931F93CF93BE
:1030A000DF93EC010E949F11182F0E946431882346
:1030B00021F081E08D838FE71CC00B818A81080F8E
:1030C000123031F0143039F4CE010E94131803C0CD
:1030D000CE010E94FF178B819A81890F081711F08A
:1030E00081E08D838D81882319F0CE010E94201804
:1030F000812FDF91CF911F910F910895EF92FF9251
:103100001F93CF93DF931F92CDB7DEB77C0181E091
:10311000F701858311E0C70169830E944D18698119
:10312000811102C0F7011682F7019681911108C042
:10313000883031F481E0868383819281890F09C0D0
:10314000662311F0F7011583813029F79111E3CF40
:103150008FEF0F90DF91CF911F91FF90EF90089527
:103160000F931F93CF93DF93EC018B0150E00E94EC
:1031700068124AE3B801CE01DF91CF911F910F9100
:103180000C941412EF92FF920F931F93CF93DF933F
:1031900000D01F92CDB7DEB78C01462F09969A83D7
:1031A00089838EE08B83D801EC91F0E0EE0FFF1F56
:1031B000EF5CFD4FE590F490BE016D5F7F4FCE0157
:1031C00001960E94B018A701BE016D5F7F4FCE012E
:1031D00001960E942F1240E2BE016D5F7F4FCE012B
:1031E00001960E941412F80141815281BE016D5F67
:1031F0007F4FCE0101960E9468124FE2BE016D5FC3
:103200007F4FCE0101960E941412D80117964D915E
:103210005C911897BE016D5F7F4FCE0101960E94B1
:1032200068120F900F900F90DF91CF911F910F9127
:10323000FF90EF90089527E1289FB001299F700D1E
:10324000112464577F4F47E150E084E792E00C94EB
:10325000703927E1289FB001299F700D1124645710
:103260007F4F47E150E084E792E00C948E39DC0117
:10327000EC91B5E0EB9FF0011124E60FF11DEE0F8C
:10328000FF1FED54FD4F859194910895DC01EC9161
:1032900045E0E49FF0011124E60FF11DEE0FFF1F42
:1032A000ED54FD4F8591949117962D913C9118976F
:1032B000AC01429FC001439F900D529F900D11247D
:1032C0000895FC01A181B2812091530330915403F0
:1032D0000E94A83824E630E040E050E00E94F9382F
:1032E000293EFDEF3F074105510520F028EE3DEF57
:1032F00040E050E0C9010895FC012081213029F40B
:1033000020914F033091500309C0223029F42091BD
:103310004D0330914E0302C020E030E0FC01878174
:103320009085AC01249FC001259F900D349F900D86
:103330001124089580914B0390914C030895FC0152
:103340006081F9E06F9FB001112465597D4F49E01C
:1033500050E00C944039DC01EC91F0E0EE0FFF1FDF
:10336000EF5CFD4F859194910C941B1360E170E02C
:103370000C94AB19CF93DF93EC01888160E081114D
:1033800008C0CE010E94461967E00E94A71587E099
:1033900011C0CE010E94461965E00E94A7158FE278
:1033A0000E94A0138F8198850E94BC1283E40E9422
:1033B000A01388E0DF91CF91089566E0FC0183813E
:1033C00094810E94A31586E0089566E0FC01858142
:1033D00096810E94A31586E00895FC018181928167
:1033E000883EFDEF9F0729F487E292E00E944F1389
:1033F00003C067E00E949F1588E0089527E1AC01B3
:10340000249FC001259F900D11248B569F4F089536
:103410000F931F93CF93DF93CDB7DEB7A4970FB66B
:10342000F894DEBF0FBECDBF8C01AB01BC01CE0155
:1034300001960E946A1BCE0101960E94D81B87E16B
:10344000FE013C96D80101900D928A95E1F7A49671
:103450000FB6F894DEBF0FBECDBFDF91CF911F91A5
:103460000F910895FC012081260F283010F420834D
:1034700002C0FC0110820C949F1961E00E94461961
:103480009C0140E050E060E870EF8AEF92E00E941B
:10349000F938293883E138074105510520F028E83B
:1034A00033E140E050E0C901089561E00E9446190F
:1034B0009C0140E050E060E47BE48CE490E00E94FA
:1034C000F938213D87E038074105510520F020ED0E
:1034D00037E040E050E0C90108950F931F93CF9368
:1034E000DF9300D0CDB7DEB78C0169837A830E9469
:1034F0003D1AAC0169817A81C80103960F900F9043
:10350000DF91CF911F910F910C9484290F931F93FA
:10351000CF93DF9300D0CDB7DEB78C0169837A8378
:103520000E94551AAC0169817A81C80105960F90F5
:103530000F90DF91CF911F910F910C948429DC01A2
:10354000EC91BAE0EB9FF0011124EB54FD4F659133
:10355000749184ED92E60E94E538CB0108950F93B3
:103560001F93CF93DF9300D0CDB7DEB78C01698373
:103570007A830E949F1AAC0169817A81C8010796FB
:103580000F900F90DF91CF911F910F910C94842990
:10359000CF93DF93EC010E949F1A2F813885821709
:1035A000930710F498878F83CE010E943D1A2B81D8
:1035B0003C818217930710F49C838B83CE010E9479
:1035C000551A2D813E818217930710F49E838D83B7
:1035D000DF91CF910895CF93DF93EC0148EE5DEF3B
:1035E00001960E94842989819A819C838B832881FA
:1035F000233039F49C0136952795369527953C83E1
:103600002B839E838D83CE01DF91CF910C94C81ABA
:10361000DF92EF92FF920F931F93CF93DF9300D02F
:103620001F92CDB7DEB749E050E061EA72E084E76F
:1036300092E00E94403984E792E00E94C81A00E0BC
:1036400010E05EE0D52E6DE7E62E62E0F62EDB821E
:10365000FA82E98241E0400FBE016D5F7F4FCE01EB
:1036600001960E94B018C8010E9429190F5F1F4FD0
:103670000032110561F70F900F900F90DF91CF91FD
:103680001F910F91FF90EF90DF900895262F443007
:1036900019F06FEF7FEF02C061E070E0223089F037
:1036A00028F4222341F0213049F00895233061F0BD
:1036B000243069F008950B960C94321A0B960C94F2
:1036C000AF1A0B960C94EB1A0B960C946D1A0B9682
:1036D0000C94861AEF92FF920F931F93CF93DF9370
:1036E000EC018B017A0164E173E00E9490178FEF87
:1036F000898786EA90E09983888387E1F801DE0173
:103700001B9601900D928A95E1F7FBA2EAA2DF9148
:10371000CF911F910F91FF90EF9008950F931F93FA
:10372000CF93DF93CDB7DEB728970FB6F894DEBFFF
:103730000FBECDBF8C01BC016C5E7F4F29E033E032
:103740004EE050E0CE0101960E942111CE0101967B
:103750000E942C1181E0F801858328960FB6F89419
:10376000DEBF0FBECDBFDF91CF911F910F910895A6
:10377000CF93DF93EC016AA17BA16F5F7F4F0B9624
:103780000E94C2180E9410120E94081283E093E067
:103790000E944F130E940C126EE0CE0144960E94CC
:1037A000E7120E94D12983E0DF91CF910C947F3101
:1037B000DF92EF92FF920F931F93CF93DF93CDB7DA
:1037C000DEB767970FB6F894DEBF0FBECDBF8C0192
:1037D00087E1D82EC8010B967C0160E0C8010E94E9
:1037E0007E1887FD2AC0853031F0863041F4C8014B
:1037F0000E948E1BF2CFC8010E94B81BEECFF701CA
:10380000DE0111969D2D01900D929A95E1F7682F9A
:10381000C8010E94A817811109C0FE013196D70185
:103820008D2D01900D928A95E1F7D7CF83E00E940C
:103830007F31C7010E94C81AD0CF67960FB6F8949F
:10384000DEBF0FBECDBFDF91CF911F910F91FF90D3
:10385000EF90DF9008951F93CF93DF93EC01162F25
:103860000E948317CE0109960E94DA29882311F05D
:10387000298501C02FEF332727FD3095812F90E058
:103880002817390719F11230C1F048F4112381F0DB
:103890001130E1F4CE010B960E94BA1917C0133013
:1038A00089F0143099F4CE010B960E94E5190EC0F0
:1038B000CE010B960E94B61909C0CE010B960E944C
:1038C000ED1904C0CE010B960E94DD1980E0DF9156
:1038D000CF911F910895CF93DF9300D0CDB7DEB77E
:1038E00089839A830E94081289819A810E944F13CA
:1038F0000E940C128091D4029091D5020E94493905
:10390000892B51F08FEE93E00E944F138091D402E7
:103910009091D5020E944F130F900F90DF91CF919D
:103920000C94B4138091470390914803892BA1F024
:103930008CE10E94950865E02AE0AC01249FC0015B
:10394000259F900D11240E9442158DE60E94A01320
:1039500083E40E94A01304C088ED93E00E944F13FB
:103960000C94B4138AE10E94950865E00E94421508
:103970008DE60E94A01386E50E94A0130C94B41358
:1039800090E0880F991F62E089599B4F0C941B139C
:103990000F931F93CF93DF9361E084E792E00E943F
:1039A00046198C0162E084E792E00E944619EC011E
:1039B00083E10E9495088017910790F4C817D907F2
:1039C00088F49C012C1B3D0BC8018C1B9D0B64E6ED
:1039D00070E00E94E538C9010E94E538862F03C0D7
:1039E00084E601C080E0DF91CF911F910F9108958F
:1039F000613011F40C94710D0C949126CF93DF93E8
:103A0000D82FC62F8EE18D0F0E942809882351F0F0
:103A10006C2F8D2F0E94F81C46E06C2FDF91CF9108
:103A20000C94691580E694E0DF91CF910C944F13CC
:103A30000F931F93CF93DF93C82F162F0E94081266
:103A40000E943A0D811108C083E090E00E94480E68
:103A5000882341F080E209C080914902882321F047
:103A600082E403C08DE601C082E60E94A01380912B
:103A700063028823C9F0D0E001E080916402D81786
:103A800031F080916302802321F081E303C08FE550
:103A900001C080E30E94A013000FDF5FD63069F7FA
:103AA00080E20E94A01303C087E00E94A513D1E02A
:103AB000DC0F8D2F0E94CD138AE30E94A013C11149
:103AC00008C00E944C23882321F00E945B23892B8D
:103AD00029F5612F8C2F0E94FE1C0E94B4130E94B6
:103AE0000C1202E00C0F802F0E94CD138AE30E947B
:103AF000A013612F8D2F0E94FE1C83E08C0F0E946B
:103B0000CD138AE30E94A013612F802F0E94FE1C18
:103B1000DF91CF911F910F910C94B4138BE594E03A
:103B20000E944F13DACF88E10E94950868E00E9456
:103B30009F1580E20C94A0130E94081284E792E083
:103B40000E94611968E00E949F1580E20E94A01304
:103B50000E947A2667E00E94A3150E94B4130E9477
:103B60000C1282E594E00E944F1367E080913703C6
:103B7000909138030E94A7150C94B4130F931F93D0
:103B800060919602709197028091980290919902AB
:103B900020918B02222371F00E94E128009196026D
:103BA000109197022091980230919902601B710B3D
:103BB000820B930B28EE33E040E050E00E94F9388E
:103BC000C9011F910F9108950E94FC22811110C01C
:103BD0000E944C23882331F00E94FC2281110AC0EC
:103BE00084E40BC00E943A0D811106C08EE405C02A
:103BF00083E403C085E401C082E40E94A01380E254
:103C00000E94A0130E94BE1D0E94281580E20C9401
:103C1000A0130E9408120E94931D67E086E10E9493
:103C20001E0D0E94B4130E940C120E94E41D67E056
:103C300083E10E941E0D0C94B4130E94E12860934E
:103C40009602709397028093980290939902109233
:103C50009202109293021092940210929502109286
:103C60008E0210928F02109290021092910281E0C7
:103C700080938B0208950F931F930E94E128009177
:103C80009602109197022091980230919902601B40
:103C9000710B820B930B6093960270939702809343
:103CA00098029093990210928B021F910F910895A0
:103CB0000E94022381111DC00E945223811119C04C
:103CC0000E943A0D882351F18091920290919302C3
:103CD000A0919402B091950280599F4FAF4FBF4F72
:103CE0008093920290939302A0939402B0939502D2
:103CF000089580918E0290918F02A0919002B091D0
:103D0000910280599F4FAF4FBF4F80938E02909387
:103D10008F02A0939002B0939102D2CF0895CF92D8
:103D2000DF92EF92FF920E94081287E494E00E94D3
:103D30004F130E94BE1D0E9428150E940C1284E49D
:103D400094E00E944F1360919202709193028091CF
:103D500094029091950238EEC32E33E0D32EE12CDD
:103D6000F12CA70196010E94F938C9010E9428157B
:103D700081E494E00E944F1360918E0270918F0253
:103D80008091900290919102A70196010E94F938CA
:103D9000C901FF90EF90DF90CF900C9428150E94FE
:103DA000081288E394E00E944F130E949B2668E06B
:103DB0000E94AB150E94B4130E940C1282E10E9473
:103DC0002809882349F08FE294E00E944F130E9453
:103DD000A12668E00E94AB150C94B4130E9408124F
:103DE00087E294E00E944F1367E086E00E941E0D78
:103DF0000E94B4130E940C128FE194E00E944F13B2
:103E000047E061E080915503909156030E94691547
:103E10000C94B4130E94081288E194E00E944F139E
:103E200067E080E00E941E0D0E94B4130E940C12F5
:103E300081E194E00E944F1367E082E10E941E0D31
:103E40000C94B4130E9408128BE094E00E944F136C
:103E50008091470390914803892B29F065E087E022
:103E60000E941E0D04C089E094E00E944F130E943E
:103E7000B4130E940C120C94B4130F931F93CF939E
:103E8000DF9300D0CDB7DEB78B0189839A830E9480
:103E900010120E94081289819A810E944F130E9479
:103EA0000C12C8010F900F90DF91CF911F910F91CD
:103EB0000C944F1388EF93E00C946B1C81EE93E00D
:103EC0000C946B1C0E9408120E94931D0E94921C6D
:103ED0000E940C120E94E41D0C94B21C0E94081255
:103EE0008FEC93E00E944F1367E08BE10E941E0D60
:103EF0000E94B4130E940C1285EC93E00E944F13B1
:103F00000C94B21C0E9408128FEB93E00E944F1396
:103F10008091470390914803892B41F069E080919B
:103F20001401909115010E944D1504C086EB93E099
:103F30000E944F130E94B4130E940C128CEA93E06B
:103F40000E944F130C94921C6CE973E08FE893E08D
:103F50000C943D1F0E94A41F0C94D12964E873E0C7
:103F600083E793E00E943D1F88E893E10C94F128D9
:103F70000E94081282E693E00C944F13CF930E94A4
:103F8000081264E070E084E792E00E94AB1980E2DE
:103F90000E94A01384E792E00E94BA1980E20E9476
:103FA000A0138091D6020E94C01C0E940C120E9495
:103FB000C81C90E08436910569F48CE892E00E9478
:103FC000DA29882321F084E00E94A5130AC08DE538
:103FD00093E005C062E00E943F158AE593E00E94ED
:103FE0004F138CE892E00E94DA29882319F0C091DF
:103FF0008C0201C0CFEFC0FF05C065E080E00E94E9
:104000001E0D03C085E00E94A51380E20E94A0134C
:104010008091740284508430A8F4C1FF05C065E02B
:1040200082E10E941E0D03C085E00E94A513C2FF1D
:1040300005C00E944A09CF910C94CD1380E2CF9124
:104040000C94A01366E080917502909176020E9414
:104050009F15CF910C94B41390918D029F5F909314
:104060008D0290E0FC013197EF30F10528F5E65D17
:10407000FF4F0C943A390C94091E0C949C1D0C941F
:104080008F1E0C94221F61E005C061E083E00C9458
:10409000181D64E080E0FBCF64E0F8CF0C94BE1FF5
:1040A0000C94CF1E0C940A1F0C94EE1E0C946E1FE1
:1040B0000C94821F0C94621F08958FEF80938C02E2
:1040C00008950F931F93CF93DF930E942423C091F1
:1040D0007702D091780261E084E792E00E9446196D
:1040E0008C01CE0165E070E00E94E5388FE00E940F
:1040F000BE0CEC0140E0BC01C8010E94C5268FE067
:104100000E94D926CE01DF91CF911F910F910C947F
:10411000102381E00C9432230E948B09882321F024
:104120000E940B230C948027089510929A020C94FD
:104130006120CF93DF930E948C200E948609EC01BE
:1041400080919A02811111C062E084E792E00E949E
:1041500046198C179D0748F481E080939A0280915C
:104160007702909178020E941E230E948B09882377
:1041700081F064E084E792E00E9446198C179D0765
:1041800040F48EE894E09093D5028093D40281E0CD
:104190002EC08091200190912101029738F18091E9
:1041A0009B02882389F08AE10E949508EC0184E74C
:1041B00092E00E947C19D195C195D1098C179D0779
:1041C0001CF48AE894E0DFCF80919C02882371F090
:1041D0008CE10E949508EC0184E792E00E949A1914
:1041E0008C179D071CF484E894E0CDCF82E0DF912A
:1041F000CF91089580939C0260939B0208957093E1
:10420000A00260939F0290939E0280939D02089566
:104210000F931F93CF93DF93C0919D02D0919E0285
:10422000CE010E94800F8C010E948609C817D90711
:1042300038F4C801DF91CF911F910F910C94620F58
:1042400081E0DF91CF911F910F91089581E00E944D
:1042500092230C940E0E0E9484230E94C40D10928F
:10426000A10280E10C94D9260F931F93CF93DF9383
:104270000E940821182F0E945B23EC010E948B09E9
:10428000882311F001E001C0012F8091A102882351
:1042900029F0BE01812F0E94312701C0812F882380
:1042A00029F081E00E94922381E00CC0002349F0B4
:1042B000BE01812F0E944D288C179D0711F00E948E
:1042C000772382E0DF91CF911F910F910895BC0178
:1042D00080E10E94BE0C0C9469260F931F93CF932C
:1042E000DF938C01EB010E94FF20BE0180E10E9460
:1042F000BE0C40E0BC01C8010E94C526CE016AE0A8
:1043000070E00E94E538CB01DF91CF911F910F91B2
:104310000C94672181E00E9432230C940E0E0E94BF
:10432000C40D0E9424238FE00C94D9260F931F9371
:10433000CF93DF931F92CDB7DEB78C018FE0498317
:104340000E94BE0C4981BC01C8010F90DF91CF9142
:104350001F910F910C94C526BC018FE00E94BE0CEA
:104360000C9469260F931F93CF93DF93C09137036B
:10437000D0913803CE010E94800F8C010E948609E3
:104380008C179D0738F4C801DF91CF911F910F91D1
:104390000C94440F81E0DF91CF911F910F9108950C
:1043A0001F93CF93DF930E94B221182F0E940B23FB
:1043B000EC01BC01812F0E943127882329F081E084
:1043C0000E94322381E019C00E948B09811107C02D
:1043D000111105C0CE010E948226882369F00E9437
:1043E0003A0D811109C0BE01812F0E944D288C1702
:1043F0009D0711F00E94102382E0DF91CF911F9161
:1044000008950E948A210E9426210C940E0ECF93BB
:10441000DF931F92CDB7DEB79091A302913039F0B0
:1044200018F0923039F00FC00E94D0210CC00E94C9
:10443000342109C00E94150F823089F089830E94BF
:10444000012289810CC0813051F49091A2029923FC
:1044500031F082E08093A3020E94C40D82E00F90AD
:10446000DF91CF9108950E94C40D8091A402909194
:10447000A5020E94800F0E94620F882329F00E94EB
:104480008F211092A30208950E942B2181E0809336
:10449000A1028093A30208958093A20208950F932E
:1044A0001F93CF93DF93EC018A019093A502809331
:1044B000A40240E00E949621B801CE01DF91CF9185
:1044C0001F910F910C946D210E94842387E08093AB
:1044D0008C0282E080938D020E94783183E0809389
:1044E000A7020895FF920F931F93CF93DF9380E06D
:1044F0000E94280901E008278091A602882381F004
:104500000E944A0990917B02FF24F394981301C002
:10451000F12C11E0811110E0913021F4112311F000
:1045200010E0F12C82E10E9428098823A9F082E1A1
:104530000E949508EC0180E00E949508C817D907F1
:1045400028F49C012C1B3D0BE90102C0C81BD90BB0
:10455000C53FD14008F001E0F11002C087E001C082
:1045600083E080938C02112329F080918C02825089
:1045700080938C02002329F080918C0281508093DB
:104580008C02F11004C0111102C0002311F081E06F
:1045900001C088E00E947F310E947311811102C026
:1045A0001092A702F11008C0111106C0011104C039
:1045B0000E947311883041F08091A702823011F47B
:1045C00081E008C082E006C08091A7028F5F8093DF
:1045D000A702F2CFDF91CF911F910F91FF90089525
:1045E00081E00E9492238FEF80938C0288E00C94EC
:1045F0007F318093A602089581E09091AA029111E3
:1046000080E0089581E02091A8023091A902232B37
:1046100009F480E008958091A8029091A90208957C
:10462000893E2DEF920710F088EE9DEF9093A9023E
:104630008093A8020E9490060C94CF0ABC018FE0E0
:104640000E94BE0C0C9410238091AA02882349F08A
:1046500080E090E00E94102381E00E94AB0610925F
:10466000AA020895CF93C82F8091AA0281110BC08E
:10467000CC2349F080E090E00E94102380E00E946B
:10468000AB06C093AA02CF91089580E090E00E940B
:10469000102381E00C94322381E09091AF029111BC
:1046A00080E0089581E02091AD023091AE02232B8D
:1046B00009F480E008958091AD029091AE020895D2
:1046C000482F8091AB029091AC022091AD023091C5
:1046D000AE028217930711F4442341F09093AE0287
:1046E0008093AD020E9457070C94CF0A0895813041
:1046F00020E4920710F080E090E49093AC02809365
:10470000AB0281E00C9460238091AF02882349F0D2
:1047100080E090E00E94772381E00E949E06109244
:10472000AF020895CF93C82F8091AF0281110BC0C3
:10473000CC2349F080E090E00E94772380E00E9443
:104740009E06C093AF02CF91089580E090E00E9452
:10475000772381E00C94922308958091740287302E
:1047600051F09CEF980F943048F08150823048F41B
:1047700082EC92E0089589EB92E008958BEC92E050
:10478000089580EB92E008958EEA94E0909367029A
:104790008093660290917402945081E0943008F006
:1047A00080E00E94F92261E08BE695E00E94E00F34
:1047B00091E0813009F090E0892F08950F931F93C5
:1047C000CF93DF930E944C220091790210917A02DC
:1047D000C0917702D091780263E084E792E00E9472
:1047E0004619A801BE010E944F2288EA94E09093E6
:1047F00067028093660260E080E795E0DF91CF91E9
:104800001F910F910C94E00FEF92FF920F931F9363
:10481000CF93DF938C01C7E7D2E0E880F98061E0B5
:1048200084E792E00E94461940E0B7010E94962179
:1048300088819981B8010E94E538CB010E94AC21A2
:1048400082EA94E0909367028093660260E08DE8CC
:1048500095E0DF91CF911F910F91FF90EF900C9415
:10486000E00FCF93DF93C0917702D091780261E09F
:1048700084E792E00E94461941E0BE010E94962121
:1048800082EA94E0909367028093660260E08DE88C
:1048900095E0DF91CF910C94E00F81E020914703E8
:1048A00030914803232B09F480E061E00E94FA2054
:1048B00086E994E0909367028093660260E082EA62
:1048C00095E00C94E00F62E084E792E00E944619C4
:1048D0006091790270917A02E0917B02F0917C0202
:1048E0004091570350915803E49F9001E59F300D8C
:1048F000F49F300D1124820F931F0E946D218CE9CB
:1049000094E0909367028093660260E08CE795E004
:104910000C94E00FCF93DF93C0917902D0917A028B
:1049200062E084E792E00E944619BE010E946D2178
:104930008CE994E0909367028093660260E089E9D5
:1049400095E0DF91CF910C94E00F84EA91E0909391
:1049500067028093660260E088E895E00C94E00FBF
:10496000CF93C82F8093D60224EB34E03093D50246
:104970002093D4028D3030F4E82FF0E0E655FF4F5D
:10498000808101C080E0809367000E94C4320E9451
:10499000EE0A0E94C423882361F184E00E947F31E3
:1049A0008C2F90E08D30910510F5FC01E75CFF4FF6
:1049B0000C943A398AE090E008C00E94A52419C0FE
:1049C0000E94632416C085E090E00E94042411C078
:1049D00080E001C081E00E94DE230BC00E944D24D4
:1049E00008C00E948A2405C00E94312402C00E948F
:1049F000AA1F0E94FD0ACF910C94A1340F931F931C
:104A0000CF93DF93EC010E941B190E94AD238C0110
:104A100060E0C8010E947E1887FD29C09091740251
:104A2000E82FFF27E7FDF095973019F4EF52FB4F81
:104A30000FC08CEF890F843018F4EB51FB4F08C086
:104A40009150923018F4E054FB4F02C0EB54FB4FEE
:104A500084918D3049F4BE0184E792E00E94081AE7
:104A6000CE010E942919D1CF0E94B024D1CFDF916D
:104A7000CF911F910F9108956DEE74E08BEC92E051
:104A80000E94901765EC74E082EC92E00E9490170F
:104A900067ED74E089EB92E00E94901768EB74E098
:104AA00080EB92E00C949017FC01428153814115F8
:104AB000510591F0A081B181B7FF03C0B195A195D7
:104AC000B10928EE33E00E94B7389A0140E050E087
:104AD0000E94F938C901089580E090E008950F938D
:104AE0001F93CF93DF9300D000D0CDB7DEB78C01FA
:104AF000862FF801628173810E94180B9C838B833F
:104B0000F801808191819A838983CE0101960E9468
:104B100054250F900F900F900F90DF91CF911F9120
:104B20000F9108950F93FC01CB01002341F046172C
:104B3000570708F4CA016417750748F407C06417DB
:104B4000750708F4CA014617570708F4BA01978396
:104B50008683918380831382128215821482338725
:104B60002287681B790B718760870F910895FC017C
:104B70009B0140E050E086819781281B390B410959
:104B80005109A285B3850E94BE382085318544270E
:104B900037FD4095542F0E941B392115310581E0C6
:104BA0004807510524F457FD05C0C90108958FEF4A
:104BB0009FEF089580E090E00895DF92EF92FF92DA
:104BC0000F931F93CF93DF93EC012A813B8124172E
:104BD000350720F4FA01E21BF30B03C0F901E41BD3
:104BE000F50B8C819D81969587958E179F0770F5A3
:104BF000888199818617970720F4FB01E81BF90B40
:104C000003C0FC01E61BF70BEF2B01F1241735075E
:104C100038F48A01021B130B7B01E81AF90A06C05B
:104C20007C01E61AF70A8901041B150BC7010E94D3
:104C30002729D82E888599850E942729D81206C051
:104C40001D830C83F986E8861B870A87DF91CF9145
:104C50001F910F91FF90EF90DF9008950F931F9396
:104C6000CF93DF93EC018B019A01A885B9850E944F
:104C7000B7382A853B8540E050E00E941B39C801C7
:104C8000A0E0B0E082179307A407B5071CF41F82C9
:104C90001E8204C0021B130B1F830E83DF91CF9172
:104CA0001F910F910895EF92FF920F931F93CF934F
:104CB000DF93EC018B017A010E94DD25A701B80189
:104CC000CE01DF91CF911F910F91FF90EF900C9447
:104CD0002E2690933E0380933D0308958091D90240
:104CE000813029F480913D0390913E03089580E046
:104CF00090E008956091390370913A038091DB024E
:104D00000C94180B2091DE02213041F041E02091FB
:104D10003D0330913E038217930708F040E0842F53
:104D200008952CE0829FC00111246091DB0289511B
:104D30009D4F0C946F256091DB028FE293E00C9401
:104D40006F25CF93DF9300D000D0CDB7DEB780E0E2
:104D50000E9495089A83898382E10E94950829819F
:104D60003A81281B390B3A83298386E10E949508F2
:104D70009C838B83CE0101960E9454250F900F9047
:104D80000F900F90DF91CF91089590933803809307
:104D9000370370933A0360933903CB016AE070E004
:104DA0000E94E53870933E0360933D034093DA021E
:104DB0000895EF92FF920F931F93CF93DF9391E0AB
:104DC0009093D902FF24F3948F3009F0F12C809353
:104DD000DB0268EC70E00E94BE0C90933C03809371
:104DE0003B030E94860920913D0330913E03409190
:104DF0003703509138030F2DBC0187E293E00E94E6
:104E000092250E94370D8093DC02809137039091A8
:104E100038030E94800FEC0110E08CE0E82E8091B6
:104E2000DC02181798F4812F0E94710DBC012091AB
:104E30003D0330913E03E19EC00111240F2DAE01D0
:104E400081529D4F0E9492251F5FE9CF1092DE0292
:104E50001092DD02DF91CF911F910F91FF90EF90A3
:104E600008950F931F93CF93DF93082FEB01809149
:104E7000DA028823C9F040913B0350913C03209112
:104E80003D0330913E032417350708F49A012C178F
:104E90003D0710F4109262028091DE02813021F011
:104EA0000E94150F8093D9028091D902813011F5AB
:104EB0008091DE02823041F411E020913D03309177
:104EC0003E03C217D30708F010E00E946E268C172D
:104ED0009D0770F0111102C0002351F09091DD0286
:104EE00081E0890F8093DD0281E09A3020F402C0D6
:104EF0001092DD0280E0DF91CF911F910F91089514
:104F00000F931F93CF93DF93EC010E948609AE01AC
:104F1000BC0187E293E00E94532610E00CE08091F0
:104F2000DC02181770F4812F0E94710DBC01019FE3
:104F3000C0011124AE0181529D4F0E9453261F5F74
:104F4000EECFDF91CF911F910F910895CF92DF9215
:104F5000EF92FF920F931F93CF93DF9360913703EC
:104F60007091380387E293E00E94B7258C0180910D
:104F70003703909138030E94800F7C01D12C9CE074
:104F8000C92E8091DC02D81698F4CD9CE001112442
:104F9000C152DD4FB701CE010E94B725081719078E
:104FA00028F0B701CE010E94B7258C01D394E9CF38
:104FB000C801DF91CF911F910F91FF90EF90DF908B
:104FC000CF9008950F931F93CF93DF93EB018093BE
:104FD0003503909336032091390330913A038C01C5
:104FE0002817390708F489010E946E268017910757
:104FF00008F4C801C817D90711F12091DE02223048
:10500000A9F48C179D0790F020913D0330913E0349
:105010002C173D07A0F040913303509134032091A9
:105020003F02309140024217530749F020913F025E
:1050300030914002309334032093330301C0CE01FA
:10504000DF91CF911F910F9108950F931F93CF93ED
:10505000DF93EC010E948609909328038093270335
:10506000D0932A03C093290310E00CE08091DC0266
:10507000181770F4812F0E94710D019FF001112407
:10508000E152FD4F91838083D383C2831F5FEECFB4
:10509000DF91CF911F910F9108951F93CF93DF93CD
:1050A000182FEB01CB010E948027CE010E942528FA
:1050B0000E94A6279093D8028093D702BE010E9437
:1050C000E2272091DE02211110C0112389F0809186
:1050D000DA02882321F00E94070E1092620281E01A
:1050E0008093DE0280E090E003C022E02093DE02A5
:1050F000DF91CF911F91089560913F03709140031C
:105100008091410390914203089512BE8DE78CBFB8
:1051100088E083BF83B7836083BF89B7826089BF1C
:10512000089580913F0390914003A0914103B09175
:1051300042030196A11DB11D80933F03909340034C
:10514000A0934103B093420308950E9491280E94C6
:1051500050320E94F4290E9403058091680081501A
:1051600019F080936800089581EE809368000E9492
:10517000AC230E945A090C94581E1F920F920FB62E
:105180000F9211242F933F934F935F936F937F93CD
:105190008F939F93AF93BF93EF93FF930E94A528A4
:1051A000FF91EF91BF91AF919F918F917F916F91FF
:1051B0005F914F913F912F910F900FBE0F901F90D5
:1051C00018952FB7F89460913F0370914003809138
:1051D0004103909142032FBF9695879577956795E8
:1051E0000895CF92DF92EF92FF92CF93DF93EC017D
:1051F0000E94E1286B017C01CC0EDD1EE11CF11C3C
:105200000E94E1286C157D058E059F05C8F3DF918E
:10521000CF91FF90EF90DF90CF90089540E0FC0198
:10522000259134910296232B11F04F5FF8CF842FF4
:105230000895282F81E090E03AE0215038F0AC0149
:10524000349FC001359F900D1124F7CF089597FD2D
:1052500002C081E008958FEF0895CF92DF92EF9220
:10526000FF92CF93611571058105910521F461E0ED
:1052700070E080E090E0C0E02AE0C22ED12CE12C6A
:10528000F12CCF5FA70196010E94F938CA01B9013C
:105290002115310541055105A1F78C2FCF91FF90C4
:1052A000EF90DF90CF900895BC0180E090E00C94E7
:1052B0002D29FC0120813181260F371F37FF03C0C4
:1052C00011821082089550E0421753071CF4518355
:1052D00040830895318320830895FC01208131812A
:1052E000260F371F121613062CF081E090E09183F1
:1052F0008083089550E0421753071CF45183408384
:105300000895318320830895DF92EF92FF920F93E7
:105310001F93CF93DF93EC018A01DD24D3941616FB
:1053200017060CF0D12CE880F980B70180E090E0FE
:105330000E942D29823028F082500E9419299C0158
:1053400002C021E030E0C701B9010E94E5380097B2
:1053500039F0DD2019F0281B390B04C09C010FC067
:10536000DD2069F0C801821B930BE816F90618F4DA
:105370002E0D3F1D01C09801398328830AC02E15C8
:105380003F0518F4E21AF30A02C0E12CF12CF9826D
:10539000E882DF91CF911F910F91FF90EF90DF9006
:1053A00008950E949F118111FCCF0E949F118823B4
:1053B000E1F30895FC01208127FD05C081818695D8
:1053C0008F5F8170089580E00895FC01208127FDA2
:1053D00009C081819FEF980F9695282F269581E02F
:1053E000921301C080E00895089508956CE87EE668
:1053F00080E00E94BE0C9093440380934303089581
:10540000CF93DF9380E00E949E0820914303309168
:1054100044032817390718F487EC95E012C086E09A
:105420000E949508EC0186E00E942809882379F003
:105430008091550390915603C817D90740F48FEB1C
:1054400095E09093D5028093D40280E02BC088E150
:105450000E949508EC0184E792E00E946119883E61
:105460002DEF920731F08C179D0718F486EB95E02D
:1054700014C08091470390914803892B11F482E076
:1054800011C087E00E9495082091490330914A039A
:1054900028173907A0F78DEA95E09093D5028093FD
:1054A000D40281E0DF91CF9108950F931F93CF93A2
:1054B000DF938C01443019F0CFEFDFEF02C0C1E081
:1054C000D0E00E947511D8011B96EC91F0E0EE0F30
:1054D000FF1FE459FE4F9C01C29FC001C39F900D66
:1054E000D29F900D112420813181820F931F9183CF
:1054F0008083DF91CF911F910F910895EF92FF92DA
:105500000F931F93CF93DF931F92CDB7DEB78C011C
:10551000443021F0EE24EA94FE2C03C0EE24E39400
:10552000F12C69830E947511D8011B96ED91FC91B5
:105530001C976981E60FF11DE491F0E0EE0FFF1F6B
:10554000E459FE4F9C01E29EC001E39E900DF29E45
:10555000900D112420813181280F391F3183208340
:105560000F90DF91CF911F910F91FF90EF900895D1
:10557000CF93DF9300D000D0CDB7DEB780E00E949C
:105580008C089A83898382E10E9495089C838B838F
:10559000AE014F5F5F4F61E080E00E94D5080F9041
:1055A0000F900F900F90DF91CF9108950F931F935D
:1055B000CF93DF93CDB7DEB728970FB6F894DEBF51
:1055C0000FBECDBF8C0189E00E948C089E838D8325
:1055D00088E00E949508800F911F98878F838AE04A
:1055E0000E948C089A8389830F8118858FE10E941D
:1055F0009508800F911F9C838B83AE014B5F5F4F9B
:1056000061E089E00E94D508AE014F5F5F4F61E025
:105610008AE00E94D50828960FB6F894DEBF0FBE28
:10562000CDBFDF91CF911F910F9108950F931F93DD
:10563000CF93DF9300D000D0CDB7DEB78C018AE0E6
:105640000E948C089A83898389E00E949508800FC4
:10565000911F9C838B83AE014F5F5F4F61E08AE0B7
:105660000E94D5080F900F900F900F90DF91CF916F
:105670001F910F91089560E070E080EE95E00E9428
:105680003D1F80E00E942809811106C00E949F11E1
:105690008130B9F780E0089581E00895CF93DF93DA
:1056A00000D000D0CDB7DEB7962F5A8349833C8314
:1056B0002B838E3121F4C9010E94D62A0DC08F316F
:1056C00021F4C9010E94162B07C0AE014F5F5F4F46
:1056D00061E0892F0E94D5080F900F900F900F90D6
:1056E000DF91CF910895FF920F931F93CF93DF9394
:1056F000F62E142F022F83E00E947F31812F0E940B
:105700009508EC0181E080933E020E945808802FAA
:105710000E948C08AC019E01602F812F0E944E2BAD
:105720000E945808FF2039F0DF91CF911F910F910F
:10573000FF900C94B82ADF91CF911F910F91FF90A9
:105740000895EF92FF920F931F93CF93DF93CDB7FE
:10575000DEB72E970FB6F894DEBF0FBECDBF0E9406
:1057600084230E943B2B882309F43FC067EF75E038
:10577000CE0101960E9490178FEF8A878BEB90E005
:105780009A83898384EF95E09D878C8786E08E8756
:1057900061E0CE0101960E947E18F82E87FD25C09B
:1057A000082F112707FD1095F801EC50FA4FE490EF
:1057B0008E2D0E942809882359F30E9458081092C0
:1057C0003E026F2DCE0101960E94A817882349F052
:1057D000F801EF50FA4F24914E2D60E08F2D0E947A
:1057E000732B81E080933E02D3CF81E00E9492230D
:1057F0002E960FB6F894DEBF0FBECDBFDF91CF91CE
:105800001F910F91FF90EF900895EF92FF920F93E9
:105810001F93CF93DF93CDB7DEB72E970FB6F894D3
:10582000DEBF0FBECDBF0E9484230E943B2B882386
:1058300059F164E776E0CE0101960E9490178FEF50
:105840008A878BEB90E09A8389838BE696E09D872D
:105850008C8789E08E8761E0CE0101960E947E18D8
:10586000F82E87FD11C0082F112707FD1095F801AC
:10587000E559F94FE49086E08F156CF38E2D0E9468
:105880002809882341F310C081E00E9492232E96BC
:105890000FB6F894DEBF0FBECDBFDF91CF911F9141
:1058A0000F91FF90EF9008950E94580810923E02C9
:1058B0006F2DCE0101960E94A817882349F0F801A8
:1058C000EC59F94F24914E2D61E08F2D0E94732BDE
:1058D00081E080933E02BFCF0E94081288ED95E0E0
:1058E0000E944F1365E080914503909146030E940A
:1058F0003F150E94B4130E940C1280ED95E00E94A7
:105900004F1367E086E10E941E0D0C94B413EF92D2
:10591000FF920F931F93CF93DF93082F10924603AC
:1059200010924503811105C00E942423CAE7DFE3DA
:1059300004C00E948423C0E0D0E20E943B2B81116E
:1059400002C0C0E04AC0F12C6AE0E62E0E946C2C36
:105950000E949F11182F0E9475119C01E29EC001A8
:10596000E39E900D1124143079F440914503509139
:1059700046034C175D0750F79C01240F351F3093E9
:105980004603209345030FC01230C1F440914503F4
:105990005091460348175907C8F2481B590B5093BA
:1059A00046034093450380914503909146030111BE
:1059B00003C00E94102302C00E947723183021F4F4
:1059C000FF2021F2C1E009C0111103C0FF24F394AC
:1059D000BDCF113009F0BACFB4CF81E0011103C0BF
:1059E0000E94322302C00E9492238C2FDF91CF911C
:1059F0001F910F91FF90EF900895DF92EF92FF9229
:105A00000F931F93CF93DF9300D000D0CDB7DEB7B5
:105A1000162F7A01D22E0E94872C8823E9F083E08A
:105A20000E947F31FC82EB828D2D0E948C089A832C
:105A30008983AE014F5F5F4F612F8D2D0E94D50886
:105A4000802F0E948C089A838983AE014F5F5F4F3D
:105A5000612F802F0E94D5080F900F900F900F900C
:105A6000DF91CF911F910F91FF90EF90DF900895FC
:105A70000F93CF93DF93CDB7DEB729970FB6F89486
:105A8000DEBF0FBECDBF6CE476E0CE0101960E9472
:105A9000901760E0CE0101960E947E1887FD0EC02F
:105AA000811103C042E350E002C048EE53E00FE032
:105AB00022E0682F80E00E94FD2CEBCF29960FB6E4
:105AC000F894DEBF0FBECDBFDF91CF910F91089547
:105AD0000F93CF93DF93CDB7DEB729970FB6F89426
:105AE000DEBF0FBECDBF66E476E0CE0101960E9418
:105AF000901760E0CE0101960E947E1887FD0EC0CF
:105B0000811103C042E350E002C04CE251E000E1E9
:105B100023E0682F81E00E94FD2CEBCF29960FB681
:105B2000F894DEBF0FBECDBFDF91CF910F910895E6
:105B30001F93CF93DF9300D000D01F92CDB7DEB775
:105B4000182F6D830E948C089A838983812F0E946D
:105B500095089C838B83AE014F5F5F4F6D81812FD2
:105B60000E94D5080F900F900F900F900F90DF912B
:105B7000CF911F9108950F931F93CF93DF93CDB7CC
:105B8000DEB72C970FB6F894DEBF0FBECDBF182F2F
:105B9000062F6AE176E0CE0101960E9490178FEF02
:105BA0008A8723EC30E03A8329831C8761E0CE01A9
:105BB00001960E947E1887FD13C08111F7CF1092C5
:105BC0003E0260E0CE0101960E94A817882321F0D2
:105BD000602F812F0E94982D81E080933E02E6CFB6
:105BE0002C960FB6F894DEBF0FBECDBFDF91CF91DC
:105BF0001F910F9108951F93CF93DF93CDB7DEB719
:105C000029970FB6F894DEBF0FBECDBF182F6EE2F6
:105C100076E0CE0101960E94901760E0CE010196D9
:105C20000E947E18682F87FD04C0812F0E94BB2D23
:105C3000F4CF29960FB6F894DEBF0FBECDBFDF912B
:105C4000CF911F910895CF93DF93CDB7DEB72A97F9
:105C50000FB6F894DEBF0FBECDBF82E08093670021
:105C60006EEB76E0CE0101960E94901760E0CE01C7
:105C700001960E947E1887FD29C08A870E94C4323F
:105C80000E94EE0A8A85823099F03CF4882369F0FC
:105C90008130B9F40E94382D14C0843081F05CF05A
:105CA000853079F40E94A12B0CC00E94052C09C0FC
:105CB0000E94682D06C087E00E94FB2D02C00E9452
:105CC000AB340E94FD0A0E94A134D0CF83E08093C0
:105CD00067002A960FB6F894DEBF0FBECDBFDF91E6
:105CE000CF9108951F93CF93DF93EC01162F0E945D
:105CF0008317CE0109960E94DA29882311F089853D
:105D000001C08FEF992787FD9095612F70E086176E
:105D1000970741F0EB85FC85E60FF71F84916D85B1
:105D20000E941E0DDF91CF911F9108951F93CF9375
:105D3000DF93EC01162F0E948317CE0109960E9473
:105D4000DA29882311F0298501C02FEF332727FD99
:105D50003095812F90E02817390769F0111105C09F
:105D600067E08B850E941E0D06C08B850E948C0803
:105D700067E00E943F15DF91CF911F91089581E068
:105D80000C94E736CF93DF93CDB7DEB729970FB6E4
:105D9000F894DEBF0FBECDBF68E177E0CE0101967B
:105DA0000E94901760E0CE0101960E947E18882321
:105DB00039F0813019F40E94BF2E02C087FFF2CF64
:105DC00029960FB6F894DEBF0FBECDBFDF91CF91FD
:105DD0000895CF93DF93CDB7DEB729970FB6F89428
:105DE000DEBF0FBECDBF60E177E0CE0101960E941D
:105DF000901760E0CE0101960E947E18813049F034
:105E0000823051F081110BC087E493E00E94572F3C
:105E1000F0CF0E94232EEDCF0E94C22EEACF87FF43
:105E2000E8CF29960FB6F894DEBF0FBECDBFDF9145
:105E3000CF910895DC015696ED91FC915797EE0FA6
:105E4000FF1FEE0FFF1FEB5AF84F6591759185917B
:105E50009491089548E150E06EE673E087E493E0A2
:105E60000E9470390C94F52948E150E06EE673E029
:105E700087E493E00E948E390C94F52948E150E0C4
:105E800069E677E00C94403987E493E00E943E2F66
:105E90000C94342FFC01228533852630310520F007
:105EA00025E030E03387228708950C94F5290F937D
:105EB0001F93CF93DF93CDB7DEB7A3970FB6F894B8
:105EC000DEBF0FBECDBF8C01BC01CE0101960E948A
:105ED000842FCE0101960E94A12F88E1FE013C96FD
:105EE000D80101900D928A95E1F70E94342F0E940B
:105EF000F529A3960FB6F894DEBF0FBECDBFDF9194
:105F0000CF911F910F9108950F931F93CF93DF931C
:105F1000EC018B0167EB77E00E9490178FEF898788
:105F20008BEC90E09983888388E1F801DE011B9671
:105F300001900D928A95E1F7DF91CF911F910F911A
:105F40000895DF92EF92FF920F931F93CF93DF9309
:105F5000CDB7DEB768970FB6F894DEBF0FBECDBFE2
:105F60007C018C01055F1F4F88E1D82E60E0C701DE
:105F70000E947E1887FD2AC08D3039F4C8010E9426
:105F80003E2F83E00E947F31F1CFF801DE011196B0
:105F90009D2D01900D929A95E1F7682FC7010E94FF
:105FA000A817811109C0FE013196D8018D2D0190ED
:105FB0000D928A95E1F706C083E00E947F31C80107
:105FC0000E944A2FC8010E94552FD0CF68960FB665
:105FD000F894DEBF0FBECDBFDF91CF911F910F911F
:105FE000FF90EF90DF90089564E670E00E94E5383E
:105FF000CB0163E00E943F1583E40C94A01368EE8C
:1060000073E00E94E538CB0163E00E943F1586E50E
:106010000C94A013CF93DF9364E670E00E94E53800
:106020009B01EC0163E0C9010E943F158EE20E94D2
:10603000A013CE016AE070E00E94E538862F0E942E
:10604000CD1381E897E0DF91CF910C944F13DC01E1
:106050005F96ED91FC919097EE0FFF1FEB57F84F75
:10606000859194910C944F130B960E941A2F24E65D
:1060700030E040E050E00E94F93865E0C9010E943C
:106080003F1580E30E94A01380E30C94A013FC0151
:1060900024E6269FC001279F900D11242081318185
:1060A000820F931F8436910510F484E690E091836B
:1060B0008083808191818D3A964220F08CEA96E22D
:1060C000918380830895FC012AE0269FC001279FC9
:1060D000900D112420813181820F931F8A30910508
:1060E00010F48AE090E09183808380819181893EE1
:1060F000934020F088EE93E0918380830895FC0123
:1061000028EE33E0629FC001639F900D729F900D57
:10611000112420813181820F931F88352BE1920752
:1061200010F488E59BE191838083808191818133A4
:10613000954720F080E395E7918380830895FC01E3
:1061400080819181680F791F6330710518F0718328
:10615000608304C083E090E091838083808191819B
:10616000893C910520F088EC90E09183808308952C
:106170000F931F93262F443019F06FEF7FEF02C06B
:1061800061E070E0022F10E00C301105D8F5F80145
:10619000EA5BFF4F0C943A3941E00B962FC00D9605
:1061A0001F910F910C9447300F961F910F910C94F3
:1061B000633044E1419622C044E143961FC045E06C
:1061C000459602C04AEF47961F910F910C946D2996
:1061D00049961F910F910C947F3048EE53E04B96F7
:1061E0001F910F910C9484294D961F910F910C943F
:1061F0009F3044E04F9602C044E081961F910F917A
:106200000C9459291F910F9108951F93CF93DF93F9
:10621000EC01162F0E948317CE0109960E94DA29FD
:10622000882311F0298501C02FEF332727FD3095F2
:10623000812F90E02817390709F442C0412F50E020
:106240004C305105E8F5FA01EE5AFF4F0C943A39FB
:106250008B850E94971334C08D859E850E94F42FF4
:106260002FC08F8598890E940A302AC065E08989ED
:106270009A891CC065E08B899C8918C063E08D8970
:106280009E890E943F151CC065E08F89988D0E94F1
:10629000561516C0898D9A8D0E94FF2F11C066E099
:1062A0008B8D9C8D03C065E08D8D9E8D0E945F154A
:1062B00007C0CE010E94273003C0CE010E943430B7
:1062C000DF91CF911F910895CF930E94020BC82FA9
:1062D000882349F080915F03811102C00E94B81F9A
:1062E00087E00E947F31C0935F038C2FCF91089588
:1062F0000E947C28709364036093630308959091D7
:106300006003981721F0809360030C94783108950E
:1063100090916003983011F40C947F31089588E0D7
:106320000C947F319B01220F331F2817390764F02B
:10633000681779072CF4A901481B590BCA01089565
:10634000181619060CF4089580E090E008959695CB
:1063500087958531910520F46AE070E00C949231C4
:106360000E948F3180E090E008950F931F93CF93A8
:10637000DF93EC01D695C795D695C795C93CD10555
:106380002CF00E948F3180E090E00EC06AE070E057
:10639000CE010E9492318C016AE070E0CE018897B4
:1063A0000E949231800F911FDF91CF911F910F9129
:1063B000089560ED77E00E94E5386AE070E00C94A3
:1063C00092316AE070E00E94E538CB016D387105CA
:1063D00020F464E170E00C9492310E948F3180E0EF
:1063E00090E008956AE070E00E94E5389B01CB01DF
:1063F00068E270E00E94E538283B314020F464E117
:1064000070E00C9492310E948F3180E090E008950A
:106410006AE070E00E94E5389B01CB0168E270E021
:106420000E94E5382135310520F464E170E00C94D8
:1064300092310E948F3180E090E008956AE070E030
:106440000E94E5389B01CB0168E270E00E94E538CC
:10645000283B314020F464E170E00C9492310E94BA
:106460008F3180E090E008954091600350E0483023
:10647000510598F4FA01E25AFF4F0C943A390C9402
:10648000A7310C94D9310C94E1310C94F2310C9475
:10649000B5310C9408320C941E3280E090E00895DF
:1064A0000E947C282091630330916403CB01821BFE
:1064B000930B0E9434322091610330916203821762
:1064C000930731F090936203809361030C94270546
:1064D0000895CF93DF931F92CDB7DEB7E0919D046F
:1064E000F0919E04309711F4E1EAF4E0CE010196B8
:1064F0002EEB8E179F0710F02193FBCF0F90DF91AB
:10650000CF910895CF93DF9300D0CDB7DEB7209120
:106510009D0430919E042115310511F421EA34E0E7
:10652000CE010196821B930B0F900F90DF91CF91BC
:106530000895CF93DF931F92CDB7DEB720919D04CE
:1065400030919E042115310511F421EA34E0F9015E
:10655000AE014F5F5F4FCF01821B930B4E175F075A
:1065600028F060816E3B11F43196F5CF0F90DF91EA
:10657000CF91089587E493E00E941A2FAB01BC01EC
:106580008EE693E00C94BA3580916900813059F41D
:1065900080915B0390915C03892B29F00E94BA32B1
:1065A00082E0809369000895CF93C82F682F8EE60C
:1065B00093E00E948037909165039C279093650338
:1065C000CF9108958BE30C94D432CF93DF93EC01F9
:1065D0008991882319F00E94D432FACFDF91CF91AC
:1065E00008950F931F93CF93DF93CDB7DEB72B970B
:1065F0000FB6F894DEBF0FBECDBF8E010F5F1F4FE9
:106600001A87098727E02B87AC01BE01655F7F4FA2
:10661000CE0109960E946812C8010E94E5322B96AD
:106620000FB6F894DEBF0FBECDBFDF91CF911F91A3
:106630000F910895CF93DF93EC011092650384E2EC
:106640000E94D432CE010E94F1320E94E232809147
:10665000670090E00E94F1320E94E232609166038E
:1066600070916703809168039091690328EE33E08D
:1066700040E050E00E94F938C9010E94F1328EE2F8
:106680000E94D43260916603709167038091680321
:106690009091690324E630E040E050E00E94F93830
:1066A000CA01B9012AE030E040E050E00E94F93828
:1066B000CB010E94F132DF91CF910C94E2328DE058
:1066C0000E94D4328AE00C94D4328091650390E029
:1066D0000E94F1320C945F33CF93DF9381E090E01E
:1066E0000E941A33C1E5D8E0F8E0CF35DF0751F05A
:1066F000FE0184910E9495080E94F1320E94E232CC
:106700002196F2CFC0E08C2F0E9491260E94F13298
:106710000E94E232CF5FC630B1F70E949B260E94F2
:10672000F1320E94E2320E94A1260E94F1320E94C0
:10673000E232DF91CF910C946533CF93DF93D82F62
:1067400082E090E00E941A33C0E08C2FDD2319F024
:106750000E948C0802C00E9495080E94F1320E949B
:10676000E232CF5FC43289F78091630290E00E94E9
:10677000F1320E94E2320E9428068091D702909165
:10678000D8020E94F1320E94E232DF91CF910C9444
:10679000653383E090E00E941A330E9499320E9490
:1067A000F1320E94E2320E9482320E94F1320E9453
:1067B000E2320C946533CF93DF93C0915B03D091A9
:1067C0005C030E946C33C230D1056CF081E0C430B0
:1067D000D1050CF480E00E949D33229721F0DF91D7
:1067E000CF910C94C933DF91CF9108950F931F93EC
:1067F00080916900813051F10E94E1282091690067
:10680000223051F460936A0370936B0380936C039E
:1068100090936D031092690000916A0310916B03CD
:1068200020916C0330916D03DC01CB01801B910B37
:10683000A20BB30B8093660390936703A093680346
:10684000B09369031F910F910C94DB331F910F914B
:1068500008950F931F93CF93DF931F92CDB7DEB7A9
:106860008A0169830E94D4326981862F90E00E9458
:10687000F1328DE30E94D432C8010E94F1320F90B0
:10688000DF91CF911F910F910C945F331F93CF93A2
:10689000DF9300D000D0CDB7DEB78FEC90E00E9440
:1068A000E5320E945F3347E050E060E085E40E94FB
:1068B000293441E050E061E085E40E94293442E05F
:1068C00050E062E085E40E94293410E040E0612F4E
:1068D000CE0101960E94B80849815A81612F81E654
:1068E0000E9429344B815C81612F82E70E94293408
:1068F00041E0612FCE0101960E94B80849815A817A
:10690000612F81E40E9429344B815C81612F82E5F3
:106910000E9429341F5F1131C9F60F900F900F901C
:106920000F90DF91CF911F9108958EE693E00E9422
:1069300001358EE693E00E942F3660E08AE00C94E9
:10694000103880916900813029F00E94953481E0EF
:106950008093690008950E94BA320E9446340E94D2
:106960005F330E9446340E945F330C949534FC01DF
:1069700024853585F901F39580819181F901EE5FD8
:10698000FE4F20813181821B930B99270895FC01D2
:1069900084859585FC01F39540815181FC01EE5F72
:1069A000FE4F208131814217530741F00190F08161
:1069B000E02DE80FF91F808190E008958FEF9FEFA1
:1069C0000895FC0184859585FC01F39540815181F2
:1069D000FC01EE5FFE4F208131814217530771F0B9
:1069E000A081B181A80FB91F8C91208131812F5FC7
:1069F0003F4F33273183208390E008958FEF9FEF3F
:106A00000895FC0181A1882329F0A489B5898C917E
:106A100086FFFBCF11A20895CF93DF93FC0126855B
:106A20003785D901B3958D919C911197019699273E
:106A3000E901CE5FDE4F4881598184179507D9F36C
:106A40000D90BC91A02DA20FB31F6C93A685B785A6
:106A5000B39511969C938E93A689B7892C9181E06A
:106A600090E0078C02C0880F991F0A94E2F7282B48
:106A70002C9381E081A30488F589E02D80818064D6
:106A8000808381E090E0DF91CF91089508951F9277
:106A90000F920FB60F9211242F933F934F938F9322
:106AA0009F93EF93FF935A991AC04CB18091900431
:106AB000909191040196992720919204309193042A
:106AC0008217930769F0E0919004F0919104E057E8
:106AD000FC4F4083909391048093900401C08CB14B
:106AE000FF91EF919F918F914F913F912F910F9037
:106AF0000FBE0F901F9018958EE693E00E94B7345A
:106B0000892B11F00C94463508951F920F920FB601
:106B10000F9211242F933F938F939F93EF93FF93A3
:106B2000209190043091910480919204909193046B
:106B30002817390711F4559812C0E0919204F0918A
:106B40009304E057FC4F208180919204909193042C
:106B50000196992790939304809392042CB9FF9106
:106B6000EF919F918F913F912F910F900FBE0F90BA
:106B70001F901895CF92DF92EF92FF92CF93DF9301
:106B8000EC016A017B01411581EE58076105710531
:106B9000F9F0EC89FD8981E090E008A002C0880F3F
:106BA000991F0A94E2F7808360E079E08DE390E03A
:106BB000A70196010E94F938215031094109510974
:106BC0005695479537952795211580E1380798F018
:106BD000EC89FD89108260E874E88EE190E0A701FD
:106BE00096010E94F9382150310941095109569501
:106BF000479537952795E889F9893083EA89FB8994
:106C0000208319A2EE89FF89408181E090E09C01F8
:106C10000D8C02C0220F331F0A94E2F7422B4083EF
:106C2000EE89FF8940819C010E8C02C0220F331F28
:106C30000A94E2F7422B4083EE89FF8920810F8C72
:106C400002C0880F991F0A94E2F7809582238083FF
:106C5000DF91CF91FF90EF90DF90CF900895CF9389
:106C6000DF93FC0186859785DC01B395EC01CE5F4F
:106C7000DE4F4D915C91119728813981421753075E
:106C8000C1F7A689B7894C9181E090E09C01058C01
:106C900002C0220F331F0A94E2F7209524232C937D
:106CA000A689B7894C919C01068C02C0220F331F24
:106CB0000A94E2F7209524232C93A689B7892C9176
:106CC000078C02C0880F991F0A94E2F780958223EF
:106CD0008C9384859585FC01EE5FFE4F2081318188
:106CE000FC01F39531832083DF91CF9108951092B9
:106CF00071031092700388EE93E0A0E0B0E08093FF
:106D0000720390937303A0937403B09375038AED99
:106D100090E090936F0380936E0380E993E09093EB
:106D20007B0380937A0390937D0380937C0380E4BC
:106D300090E090937F0380937E0329E230E03093CC
:106D40008103209380032BE230E030938303209370
:106D500082032AE230E030938503209384039093EA
:106D60008703809386038CE290E09093890380935D
:106D7000880384E080938A0383E080938B0387E019
:106D800080938C0385E080938D0381E080938E0354
:106D900008950F931F93CF93DF9300D0CDB7DEB745
:106DA0008C0169837A830E94883969817A81861788
:106DB000970729F0C8010E94AF3981E001C080E047
:106DC0000F900F90DF91CF911F910F910895CF9366
:106DD000DF93C82F69E778E088E698E00E943D1FBE
:106DE00067E070E080E090E00E94C93681111DC02C
:106DF000C1111BC061E070E08AE890E00E94C936D2
:106E000081111BC0C11119C0D0E062E070E08CE6B6
:106E100093E00E94C936811118C0D11116C0CC234D
:106E2000F9F0DF91CF910C94AE1F85E698E00E94B7
:106E30004F130E94EB08C1E0DDCF82E698E00E948C
:106E40004F130E94081BD1E0E0CF8FE598E00E942D
:106E50004F130E94442F80ED97E00E94F128DFCF6E
:106E6000DF91CF9108950E94DF370E945F10CCE739
:106E7000D5E30E944D102097E1F30E947C35F9CFB5
:106E8000CF92DF92EF92FF920F931F93CF93DF93F6
:106E90006C017A01EB01E60EF71E00E010E0CE1562
:106EA000DF0561F06991D601ED91FC910190F081CF
:106EB000E02DC6010995080F191FF1CFC801DF9118
:106EC000CF911F910F91FF90EF90DF90CF90089599
:106ED0006115710581F0DB010D900020E9F7AD012E
:106EE00041505109461B570BDC01ED91FC9102808A
:106EF000F381E02D099480E090E008950C946837C8
:106F0000DC01ED91FC910190F081E02D09948093DA
:106F10006A0008951F920F920FB60F9211242F93BB
:106F20003F938F939F93AF93BF93809195049091DC
:106F30009604A0919704B09198043091940423E0B2
:106F4000230F2D3720F40196A11DB11D05C026E8A1
:106F5000230F0296A11DB11D2093940480939504E4
:106F600090939604A0939704B09398048091990409
:106F700090919A04A0919B04B0919C040196A11D4C
:106F8000B11D8093990490939A04A0939B04B093AD
:106F90009C04BF91AF919F918F913F912F910F9042
:106FA0000FBE0F901F9018950197009739F0880F2A
:106FB000991F880F991F02970197F1F70895789408
:106FC00083B7826083BF83B7816083BF89B78160E5
:106FD00089BF1EBC8EB582608EBD8EB581608EBDB0
:106FE0008FB581608FBD85B5846085BD85B58064B2
:106FF00085BD329A319A309A379A1AB808958430FA
:1070000039F0853049F0833051F48FB58F7702C065
:107010008FB58F7D8FBD089585B58F7D85BD089512
:10702000CF93DF9390E0FC01E055F74F2491FC01F2
:10703000E352F74F8491882349F190E0880F991F1C
:10704000FC01E25EF64FA591B4918C5E964FFC0177
:10705000C591D4919FB7611108C0F8948C91209587
:1070600082238C93888182230AC0623051F4F89481
:107070008C91322F309583238C938881822B888347
:1070800004C0F8948C91822B8C939FBFDF91CF9199
:1070900008950F931F93CF93DF931F92CDB7DEB761
:1070A000282F30E0F901ED57F74F8491F901E055B1
:1070B000F74F1491F901E352F74F04910023C9F0FF
:1070C000882321F069830E94FF376981E02FF0E077
:1070D000EE0FFF1FEC5EF64FA591B4919FB7F894A9
:1070E0008C91611103C01095812301C0812B8C9379
:1070F0009FBF0F90DF91CF911F910F910895CF9374
:10710000DF93282F30E0F901ED57F74F8491F90113
:10711000E055F74FD491F901E352F74FC491CC23D6
:1071200091F081110E94FF37EC2FF0E0EE0FFF1F6E
:10713000E65FF64FA591B4912C912D2381E090E06C
:1071400021F480E002C080E090E0DF91CF910895CB
:10715000A29FB001B39FC001A39F700D811D112498
:10716000911DB29F700D811D1124911D08950E94E3
:10717000A838B7FF0895821B930B08950E94A83882
:10718000A59F900DB49F900DA49F800D911D11247B
:107190000895DB018F939F930E94BE38BF91AF91FA
:1071A000A29F800D911DA39F900DB29F900D112461
:1071B0000895991B79E004C0991F961708F0961B53
:1071C000881F7A95C9F780950895AA1BBB1B51E1CA
:1071D00007C0AA1FBB1FA617B70710F0A61BB70B47
:1071E000881F991F5A95A9F780959095BC01CD01EC
:1071F0000895A1E21A2EAA1BBB1BFD010DC0AA1FF8
:10720000BB1FEE1FFF1FA217B307E407F50720F00F
:10721000A21BB30BE40BF50B661F771F881F991F8A
:107220001A9469F760957095809590959B01AC01D3
:10723000BD01CF010895052E97FB1EF400940E9416
:10724000323957FD07D00E94F93807FC03D04EF4BD
:107250000C94323950954095309521953F4F4F4FC2
:107260005F4F089590958095709561957F4F8F4FF2
:107270009F4F0895EE0FFF1F0590F491E02D0994A4
:10728000FB01DC0102C005900D9241505040D8F73F
:107290000895FC0105900020E9F7809590958E0FE8
:1072A0009F1F0895FB01DC014150504048F00590BC
:1072B0000D920020C9F701C01D9241505040E0F7E7
:1072C0000895FB01DC014150504048F001900D92BF
:1072D0000020C9F701C01D9241505040E0F70895C9
:1072E000DC01CB01FC01E199FECF06C0FFBBEEBB88
:1072F000E09A31960DB20D9241505040B8F7089582
:10730000E199FECF9FBB8EBBE09A99278DB308957C
:10731000A8E1B0E042E050E00C947239DC01A40F27
:10732000B51F4150504048F0CB01840F951F2E915E
:107330000E949F3941505040D0F70895262FE1997F
:10734000FECF9FBB8EBBE09A01970DB2021631F0C3
:107350002DBB0FB6F894E29AE19A0FBE08950196FC
:0E736000272F0E949F390C949E39F894FFCF7E
:10736E000000A1042000FF03E10101000040001411
:10737E00005400000001020102010101010101019E
:10738E000000050101010100000000008E10000048
:10739E0000007D174037000000008317000000003A
:1073AE00F217000000002B1C461B050608070509F6
:1073BE000905070000050700000000722E7E2A0056
:1073CE00000000962E552A000000000531B83056F8
:1073DE003D302E333200000000000C354037B734FC
:0673EE00E134C734013553
:00000001FF
